:020000040800F2
:10000000F8160020ED010008D75800080943000841
:10001000D5580008D11600080D6200080000000045
:100020000000000000000000000000008D5C0008DF
:100030005926000800000000E15900088D5F000803
:10004000070200080702000807020008070200086C
:10005000070200080702000807020008070200085C
:10006000070200080702000807020008070200084C
:10007000070200080702000807020008070200083C
:1000800007020008070200085D14000807020008C4
:10009000070200080702000807020008070200081C
:1000A000070200080702000807020008070200080C
:1000B000696000080702000807020008070200083C
:1000C0000D430008070200080702000807020008A5
:1000D00007020008070200080702000807020008DC
:1000E00007020008070200080702000800F002F8F3
:1000F00000F06CF80AA090E8000C82448344AAF156
:100100000107DA4501D100F061F8AFF2090EBAE853
:100110000F0013F0010F18BFFB1A43F0010318473B
:10012000E89D0000089E00000A444FF0000C10F803
:10013000013B13F0070408BF10F8014B1D1108BF65
:1001400010F8015B641E05D010F8016B641E01F805
:10015000016BF9D113F0080F1EBF10F8014BAD1C55
:100160000C1B09D16D1E58BF01F801CBFAD505E073
:1001700014F8016B01F8016B6D1EF9D59142D6D3CD
:10018000704700000023002400250026103A28BFF5
:1001900078C1FBD8520728BF30C148BF0B607047F9
:1001A000662907F0EE85642900F08E8000207047F4
:1001B0001FB507F0DAFD00F01DFC0400002000214F
:1001C00006F0E0FEE0601FBD10B510BD00F014FDAC
:1001D0001146FFF7EDFF06F0F5FD00F032FD03B428
:1001E000FFF7F2FF03BC00F077FD000009488047ED
:1001F00009480047FEE7FEE7FEE7FEE7FEE7FEE709
:10020000FEE7FEE7FEE7FEE704480549054A064B20
:1002100070470000915F0008ED000008F810002012
:10022000F8160020F8120020F81200200FB41CB5B8
:10023000074B06AA7B4469460090059800F0C1FB75
:100240000020694600F0D0FB1CBC5DF814FB0000E8
:10025000B107000070B50446856900683026C10604
:1002600000D42026C00708D070BDD4E90121304653
:100270009047206A00F1010020626D1EF5D570BD27
:1002800070B5044685690068C00708D170BDD4E91F
:10029000012120209047206A00F1010020626D1E9C
:1002A000F5D570BD09684A0501D540B27047C9054A
:1002B000FCD500B2704709684A0501D5C0B2704745
:1002C000C905FCD580B270472DE9F04107460025ED
:1002D00010687529394616A411D0FFF7E3FF0028EE
:1002E00003DAC0F1000013A407E039688A0701D5DA
:1002F00011A402E0490704D510A4012501E0FFF78D
:10030000DAFF00210A2307F1240607E0B0FBF3F22D
:1003100003FB1200303070541046491C0028F5D100
:100320002B4622463846BDE8F04100F0DFB8000019
:10033000000000002D0000002B0000002000000045
:100340002DE9F05F4FF0000A044689464FF0800B1C
:10035000C0F820A02046E1688847002876D02528EC
:1003600006D0D4E901219047206A401C2062F1E7C1
:10037000564F00267F442046E168884720280546DE
:1003800008DB312D06D207EB050010F8200C08B170
:100390000643F0E7B00701D526F00406C4F81CA018
:1003A0000027C4F818A02A2D09D0284606F094F991
:1003B00038B304EB8708303DC8F8185019E059F8F5
:1003C000041B204604EB87029161E1688847012FF6
:1003D000054618D1E069002820DA26F020061DE045
:1003E000D8F8180000EB800005EB40003038C8F862
:1003F00018002046E1688847054606F06DF9002898
:10040000EED1012F0AD02E2D08D12046E168884771
:100410007F1C0546022F46F02006C4DBA069002899
:1004200003DA404246F00106A061F00701D026F051
:1004300010066C2D0BD0682D09D04C2D36D06A2DAE
:1004400034D0742D32D07A2D30D017E03BE0E16803
:100450002F4620468847B84205460AD158466C2F99
:1004600001D04FF48060E168064320468847054686
:1004700004E040206C2F00D0800006431DB3A5F19E
:100480004100192802D8203546F400664A4629461C
:10049000204626604E46FFF783FE90B101280DD01E
:1004A000F61D26F0070000F1080953E74C2D5046D1
:1004B000D9D058466A2DD6D00020D4E706F10409D9
:1004C00048E728464DE7206ABDE8F09FFA9900000A
:1004D00070477047704710B500F090FA006810BD83
:1004E00010B5044600F08AFA046010BD2DE9F0470B
:1004F0000D4604469246994600F124080168880694
:1005000004D5E06921F01001216000E001200027FE
:10051000A84201DDA0EB0507A16907EB050202EB8C
:100520000300A1EB0000A0612068C00602D42046B1
:10053000FFF790FE002608E0D4E901211AF8060032
:100540009047206A401C761C20624E45F4DB2068F0
:10055000C0060AD52046FFF77DFE06E0D4E901215A
:1005600030209047206A401C2062381EA7F1010706
:10057000F4DC07E0D4E9012118F805009047206A6F
:10058000401C2062281EA5F10105F3DC2046FFF780
:1005900077FE21680220090600D40120BDE8F0871B
:1005A00070472DE9FF4F0C461E464FF0FF378DB0C8
:1005B000D2E90001DDF868800A908946C1F30A5546
:1005C00005B93D46002108464FF00000B9F1000F83
:1005D00000F4400005DA00EB80004FF4400101EA2E
:1005E00050004FEA905ABAF1010F00DDBA460A985E
:1005F00050EA490030D044F61050A5F2FF3545438B
:10060000CAF100000B902F14B8F1000F3DD07542D5
:100610000B9A291E00DC524600DA694206A800F057
:1006200075FA06AB07CB03AB07C348460A9900F03F
:100630005AFB8DE80700A0F500501F380090039882
:10064000002D25DD42F21F015246084403A9039004
:10065000684600F0B9FD24E0B8F1010F4FF000004A
:1006600001D1F24307E0302101E02154401CB042A7
:10067000FBDB30460022002121540D99C1F808808F
:10068000C1E9002011B0BDE8F08FBD1B6D1CBFE7B4
:10069000A0F5005052461F3803A90390684600F0A9
:1006A000A7FD8DE807000004000C03D04FF0FF30D9
:1006B000410800E01046B8F1000F03D0002200927C
:1006C00015461FE0751E06D400F09CF902F13002B9
:1006D00062556D1EF8D5B3460122084302D00022B0
:1006E0007F1C04E02078302801D100227F1E002AE0
:1006F000099789D01DE0112D07DA00F083F9303217
:1007000062556D1C50EA0102F5D108430FD100215A
:10071000681E05E0235C625C6354491C2254401E41
:100720008142F7DBAB46A81B401E099001E0009810
:1007300048B1002004F80B000D98099AC0F8088011
:10074000C0E9002B9EE711264FF000085CE72DE979
:10075000F04F88460446D21D22F0070191B0D1E93E
:100760000001CDE90A0105F0A3FF02460B98C10F75
:100770004FF02D0007D123682B205FEA837C02D441
:10078000202000EAC300032A099001D0072A05DBD4
:1007900003464146204600F07BF90BE120688006C5
:1007A00001D5E06900E0062011238146B8F1650F0C
:1007B00006D0B8F1660F16D0B8F1670F6ED130E0F1
:1007C0000020B9F1110F0090484600DA431C0AAA34
:1007D00001A90CA8FFF7E5FEDDE90C70002609F180
:1007E0000105834646E001204B4600904FF000474C
:1007F0000AAA01A90CA8FFF7D4FEDDE90DB00C99F7
:100800005D46002618B909F1010001EB0005B9EBBE
:10081000050003D4C0F1FF3609F10105A5EB09007D
:1008200029E0B9F1010F01DA4FF001090020B9F117
:10083000110F0090484600DC03460AAA01A90CA843
:10084000FFF7AFFEDDE90C704D46002683462068B9
:1008500000070AD4AB4500DA5D4601A8012D04DD8E
:10086000411911F8011C302907D04F4502DA17F160
:10087000040F04DA0120824610E06D1EEEE7002F1F
:1008800002DCED1B3E4403E0781CA84200DD054677
:10089000A7EB060000F1010A4FF0004720680007AF
:1008A00003D4AA4501DB4FF0FF3A0021B7F1004F16
:1008B0000DF143088DF8431022D002202B23002F86
:1008C00001DA7F422D230A22011EA0F1010000DC83
:1008D0004FB197FBF2F102FB117C0F460CF1300C8B
:1008E00008F801CDF0E7A8F101004FF045010370D1
:1008F0002268120500D46521A0F1010800F8011C4E
:1009000009980FA9A1EB080707F1070700B101201B
:1009100000EB050101EBEA70A1693844A1EB00008E
:10092000A0F10100A0612068C00602D42046FFF7B4
:1009300091FC099830B1D4E901219047206A00F177
:10094000010020622068C00620D52046FFF782FC07
:100950001CE0002E04DBB34502DD01A8805D00E051
:100960003020D4E901219047206A761C401CBAF15E
:10097000010A20620AD100F03DF8C0680168405CBD
:10098000D4E901219047206A401C2062281EA5F16D
:100990000105DEDC07E0D4E9012118F8010B9047DE
:1009A000206A401C2062381EA7F10107F3DC2046B4
:1009B000FFF766FC022065E601694A1C02610878BF
:1009C000704700B58FB0CDE901310021059105498F
:1009D0007944CDE9031011466846FFF7B1FC0FB02A
:1009E00000BD0000E5FFFFFF0A6802F8010B0A6086
:1009F0007047000000487047B4100020004870475E
:100A00009410002030B5B0F10A024FEA900E71F157
:100A100000034EEA817EB0EB0E0061EB91014FEADC
:100A2000101E4EEA017E10EB0E0041EB11114FEA51
:100A3000102E4EEA016E10EB0E0041EB11214FEA31
:100A4000104E4EEA014E10EB0E0041EB11414018E2
:100A500041F100014FEAD00040EA41704FEAD10174
:100A600010EB80054FEA810444EA907444EB0104E2
:100A70006D1944EB0404521BA3414FF0000348BF1F
:100A80000A3200D530BD401C41F1000130BD0000EC
:100A90002DE9F04104461F4603260168072A01F4A8
:100AA000006003DB15A520B915A502E015A500B966
:100AB00015A521F010002060A069C01EA0610FB133
:100AC000401EA0612046FFF7C5FB4FB1D4E90121CC
:100AD00038469047206A401C2062C01C206206E015
:100AE000206AFAE7D4E9012115F8010B9047761E38
:100AF000F8D22046FFF7C4FBBDE8F0814E414E001E
:100B00006E616E00494E4600696E66002DE9F04741
:100B1000814616468AB035487844D0E9002380687B
:100B20000092CDE90130314878440C38D0E90223F5
:100B3000006903924FF03702CDE9043041F69B3053
:100B4000014491FBF2F0A0F1800502FB10141B3C64
:100B500002D56442012000E00020DFF890A080462A
:100B60000027FA44AAF1C60A0DE0E00709D0324690
:100B7000684607EB47010AEB810100F039FB8DE87D
:100B8000070064107F1C002CEFD1184F7F44B43F46
:100B900017E0E80713D007EB04100DF1180A90E8EE
:100BA0000E00AAE80E00C068F04201D19819089022
:100BB000324606A903A800F01BFB03AB07C36D1068
:100BC000641C002DE5D132466946B8F1000F03A838
:100BD00002D000F0F9FA01E000F00AFBC9E90001D7
:100BE000C9F808200AB0BDE8F0870000E4920000D0
:100BF00000487047941000207546FFF7F9FFAE4695
:100C000005006946534620F00700854618B020B518
:100C1000FFF7FAFABDE820404FF000064FF000075A
:100C20004FF000084FF0000B21F00701AC46ACE894
:100C3000C009ACE8C009ACE8C009ACE8C0098D4601
:100C400070470446AFF300802046FFF7C8FA000063
:100C50004FF0013C50F8042B51F8043B9A4221D14B
:100C6000A2EB0C03934313EACC1317D150F8042BD7
:100C700051F8043B9A4215D1A2EB0C03934313EABB
:100C8000CC130BD150F8042B51F8043B9A4209D1F4
:100C9000A2EB0C03934313EACC13DBD04FF000001C
:100CA000704700BFD01A01BAB1FA81F101F0180102
:100CB00022FA01F0CB40C1F12001DBB2C0B2C01A70
:100CC0002CFA01F3D11A914311EAC311E6D170470E
:100CD000004870479810002001491820ABBEFEE77D
:100CE0002600020070475FEA400C08BF91F0000F39
:100CF0004FEA8C234FEAC12243EA51514FEA1C507C
:100D000018BF00F5F0404FEA300018BF41F0004135
:100D10005FEA6C5C00F02980BCF1FF3F08BF40F047
:100D200080407047130C06BF12044FF0100C4FF0B8
:100D3000000C130E04BF12020CF1080C130F04BFB9
:100D400012010CF1040C930F04BF92000CF1020C81
:100D5000D30F04BF52000CF1010C11464FF00002FA
:100D6000A0F11F00A0EB0C00704711F0004F08BF6E
:100D7000704731F000413FF4D5AF0B0C06BF0904BA
:100D80004FF0100C4FF0000C0B0E04BF09020CF1D9
:100D9000080C0B0F04BF09010CF1040C8B0F04BFEE
:100DA00089000CF1020CCB0F04BF49000CF1010CBF
:100DB000CCF12003A0EB0C0022FA03F302FA0CF2B0
:100DC00041EA030100F10100704720F07F4C80EA06
:100DD000030023F07F47ACEB070303F57C5300F0DF
:100DE000004003F1FF032DE980494FEA154B09B498
:100DF0004FEA144325EA0B4E24EA03480FF2042677
:100E000006EB132749083E785FEA320203FB0667C8
:100E1000C7F5000707FB06F64FEA54374FEAD646F8
:100E200006F1020607FB066CCCF1005C4FEA1C479A
:100E30002CEA074C07FB06F40CFB06F504EB154601
:100E40004FEA961634BF00204FF000404FEAD137EA
:100E500006FB07FC4FEA1C4C0CFB0BF7D21B03FBF9
:100E60000CF761EB07010CFB0EF7B0EB074072EBE0
:100E700017420CFB08F734BFA2EB0742B2EB074264
:100E800061EB17414FEA0C444FEA910706FB07FC60
:100E90004FEA1C4C0CFB0BF7B0EBC74072EB573220
:100EA00003FB0CF734BFA2EBC742B2EBC74261EBC6
:100EB00057310CFB0EF7B0EBC70072EB57720CFB0F
:100EC00008F734BFA2EBC702B2EBC70261EB577160
:100ED000039F4FEA816141EA921104EBCC044FEA8F
:100EE000D1374FEA826206FB07FC42EA90124FEAD2
:100EF00080604FEA1C4C0CFB0BF7D21B03FB0CF77A
:100F000061EB07010CFB0EF7B0EB074072EB1742E9
:100F10000CFB08F734BFA2EB0742B2EB074261EBD0
:100F200017414FEA8C554FEA910704EB9C2406FBCE
:100F300007FC4FEA1C4C0CFB0BF7B0EBC74072EB05
:100F4000573203FB0CF734BFA2EBC742B2EBC742E8
:100F500061EB57310CFB0EF7B0EBC70072EB577229
:100F60000CFB08F734BFA2EBC702B2EBC70261EB80
:100F7000577115EB4C254FEA816141EA92114FEA16
:100F800082624FEAD13742EA901206FB07FC44F135
:100F900000044FEA80604FEA1C4C0CFB0BF7D21B9D
:100FA00003FB0CF761EB07010CFB0EF7B0EB0740FE
:100FB00072EB17420CFB08F734BFA2EB0742B2EB0F
:100FC000074261EB174115EB1C154FEA813141EAED
:100FD00092414FEA823242EA90424FEA80304FEA31
:100FE0000C7644F1000448EA03434EEA0B484FF004
:100FF000000EB2EB080C71EB030724BF62463946C2
:101000004EEB0E0E4FF0000B0018524149414BEBD6
:101010000B0BB2EB080C71EB03077BF1000B24BF49
:10102000624639464EEB0E0E4FF0000B001852414F
:1010300049414BEB0B0BB2EB080C71EB03077BF157
:10104000000B24BF624639464EEB0E0E51EA0207F2
:1010500018BF46F0010616EB0E7655F1000254F16A
:10106000000103D5BDE88901BDE80088BDE889011C
:10107000BDE80048B619524141EB0101A3F101035B
:10108000704780807F7E7D7C7B7A797877767675F5
:101090007473727171706F6E6E6D6C6C6B6A6A696D
:1010A0006868676666656464636362616160605F07
:1010B0005F5E5E5D5D5C5C5B5B5A5A595958585780
:1010C00057565655555554545353525252515150E8
:1010D00050504F4F4F4E4E4D4D4D4C4C4C4B4B4B3B
:1010E0004A4A4A4949494848484747474746464681
:1010F00045454544444444434343434242424241BC
:101100004141002B26D4770021D01CB54FEA370788
:1011100003B44FF010004FF010014FF000000FBC6F
:10112000BDE810400BF1010BBBF1010F08BF5FEAF6
:10113000170722BF12F1010211F101014FF0004126
:1011400043F1000300F0004043EA00007047F9D388
:101150005708DAE746EA064613F1400F4FEA16460B
:101160001FDD13F1200FDFBF16430A460021203395
:101170005B42C8D0C3F1200746EA064602FA07F7E9
:101180004FEA164646EA0706C3F1200722FA03F2A1
:1011900001FA07F721FA03F14FF0000342EA0702D0
:1011A000B1E746EA020646EA06464FEA164646EA2E
:1011B0000106BCBF46EA0646360C4FF000034FF06E
:1011C00000024FF000019EE72DE9C048934630B47D
:1011D00091E8380007C831EA400C48BF34EA430CB4
:1011E00003D5FFF7F2FDFFF78CFFF0BCBDE80088E8
:1011F0002DE9C048934630B491E8380007C810F094
:10120000804F08BF13F0804F03D100F005F8FFF7BF
:1012100078FFF0BCBDE8008820F07F4780EA03003B
:1012200023F07F4C07EB0C03A3F57C5300F0004048
:10123000A3F1FE0392F0000F00F0B38095F0000FD1
:1012400000F077802DE901494FEA11404FEA14463A
:1012500021EA004800FB06FC24EA064708FB06F6E4
:1012600007FB08F800FB07F718EB06484CEB164C99
:101270004FEA124B18EB07484FEA15464CEB174064
:1012800022EA0B4E0BFB06FC25EA06470EFB06F690
:1012900007FB0EFE0BFB07F71EEB064E4CEB164C46
:1012A0004FF000061EEB074E4CEB174B18EB0B08EC
:1012B00040F1000018EB0E0B58EB000840F1000065
:1012C0008F1A4FF000013CBFC943661B14BFB5EB3A
:1012D000040C00213CBFC943F61B4FEA17444EEAF9
:1012E0008E0E27EA04454FEA1C4704FB07622CEAEE
:1012F000074C05FB07F70CFB05F604FB0CFC16EB93
:10130000074642EB174216EB0C4642EB1C421BEB26
:10131000060658EB0202414146EA9E0601D5BDE8A9
:101320000189B619524141EB0101A3F10103BDE866
:1013300001894FEA14454FEA114724EA054621EA9C
:10134000074C05FB07F406FB07F70CFB06F105FB52
:101350000CFC11EB074144EB17444FEA124711EB29
:101360000C4144EB1C4422EA074C05FB07F206FB48
:1013700007F70CFB06F605FB0CFC16EB074642EBE9
:10138000174216EB0C4642EB1C456A1854F100015B
:1013900048BF7047B619524141EB0101A3F1010367
:1013A000704795F0000F37D04FEA11424FEA1447CB
:1013B00021EA024624EA074C02FB07F106FB07F785
:1013C0000CFB06F402FB0CFC14EB074441EB174149
:1013D0004FEA154714EB0C4441EB1C4125EA074C3E
:1013E00002FB07F506FB07F70CFB06F602FB0CFCFD
:1013F00016EB074645EB174516EB0C4645EB1C4232
:10140000121951F1000148BF7047B619524141EB22
:101410000101A3F1010370474FEA14454FEA114758
:1014200024EA054621EA074C05FB07F106FB07F70E
:101430000CFB06F24FF0000605FB0CFC12EB07421A
:1014400041EB174112EB0C4251EB1C4148BF704776
:10145000921841EB0101A3F101037047104810B548
:10146000016821F0020101600E480168B1F5CE6FFC
:101470003CBF012108460CD30068A0F26F6006F063
:1014800019F8094A094B05F079FE05F0CFFFC0B203
:10149000012101F0DDF906490120087010BD0000AE
:1014A000002401404C240140A4703D0AD7A30A4007
:1014B0000000002030B522482249234C006883B048
:1014C00088420CBF4B210021A180008803F0E6FF79
:1014D00004F0C4FF05F050FBA078E17808446FF0F9
:1014E0007F0101EB500006F04DFB05F0EFFA1749C4
:1014F000886006F053FACDE90001164D2378627832
:10150000134905F12300FEF791FEA08805F123039E
:101510005D3081B2002240F2591003F065FEA088D0
:10152000EB1E5D3081B200224FF4BE7003F05CFE12
:1015300005F012F803B0BDE8304005F09BBB000099
:10154000580000205C000020E80C00206C100020F7
:10155000947E0008F60C00202DE9F041DFF84C8164
:101560005349544CD8F8000082B088420CBF4B213C
:101570000021A180008803F091FF4F4DE088298869
:10158000401AD8F8001008440079803806F0FAFABA
:1015900005F09CFA494E706106F000FACDE90001B1
:1015A0002378627846494748FEF740FEA088454BBD
:1015B000793081B2002240F2591003F015FEA08864
:1015C000414F793081B27B1C00224FF4BE7003F092
:1015D0000BFE20892988401AD8F8001008440079A9
:1015E00080380028B8BF404206F0CCFA05F06EFA09
:1015F000B06106F0D3F9CDE90001DFF8C8802378A7
:1016000062782F4908F10500FEF710FEA08808F166
:1016100005036B3081B2002240F2591003F0E4FD63
:10162000A0887B1C6B3081B200224FF4BE7003F0A7
:10163000DBFD04F037FE04F0A3FE21892888E28850
:10164000091A101A081A214900EB80008000096865
:101650004988484305F017FF05F0D6F901464FF0D9
:101660007E5006F0CDF9706206F098F9CDE90001E0
:1016700023786278124908F11400FEF7D7FDA0889C
:1016800008F11403413081B2002240F2591003F0F6
:10169000ABFDA0887B1C02B00022BDE8F0414130C8
:1016A00081B24FF4BE7003F09FBD000058000020CF
:1016B0005C000020E80C0020360000206C100020A8
:1016C000947E0008F60C0020F20C00200C00002094
:1016D000FEE7000070B504462248234D0078FD283F
:1016E0002CD0FE2818BF70BD208820490988891C8D
:1016F000814228BF70BD002101F048FA2878411CC2
:1017000029700A2820882CBF401F401E20801849BD
:1017100080B2184B0A88904203D11988891E8842EA
:1017200005DC1988884203D1911C884200D22180AF
:101730002088BDE87040012101F028BA0E492088B8
:101740000988891E8842A8BF70BD002101F01EFAD9
:101750002878411C29700A2820882CBF401D401C75
:10176000D4E700008F0E0020890F002036000020F3
:10177000EE0C0020F00C00203800002070B5AD4CBD
:101780002046E1780078FD2908BF401C03D0FE29DF
:1017900008BF401E00D1207020780025FF2804BF1C
:1017A0000A20207002D00A2888BF2570607821782E
:1017B00088421CBF002001F0AFF820780C2880F090
:1017C0003281DFE800F006234C688EA4A9D2F7F638
:1017D000F5F499486060E078FB2803D0F7280DD035
:1017E00000F021B99548457095484570012001F0F9
:1017F000F3FE95499348086000F015B99249934863
:101800000860012001F0F2FD00F00DB99048606021
:10181000002005F015F8E078F72803D0EF2808D06D
:1018200000F001B98B480068C178052929D300F080
:10183000FAB888480068C178002900F0F48028E0F0
:10184000C170844884490068C07800EB800001EBD7
:1018500040006168086105F08FF800F0E4B87F4847
:101860006060012004F0ECFFE078F72803D0EF2857
:1018700009D000F0D8B877480068C178052980F011
:10188000D280491CDCE773480068C178002900F069
:10189000CA80491ED4E772486060E178EF2902D01F
:1018A000F72918D0BFE0A1780E2938BF491C44D2CF
:1018B000A170C9B26B4B01EB810203EB42020261E2
:1018C000694830F8110069490968488004F014FB40
:1018D00004F012FAA7E0A178002918BF491E2CD005
:1018E000E6E763486060E178F72902D0FB2907D07A
:1018F00099E055495F480860012001F0F5FD92E04C
:10190000514A5D49116040F21F4141818BE05B48C3
:10191000606004F0A3FF86E05A49594860605A4B62
:101920000A689A4204D1514A1268127A012A7AD07E
:10193000E278F72A02D0EF2A11D074E0A060534871
:10194000086041495248086048480068017A012906
:1019500028D001210172084601F0E2FB22E0434851
:101960000068017A01295ED12AE046494948606051
:10197000464B0A689A4204D13C4A1268127A012AFC
:1019800051D0E278F72A02D0EF2A14D04BE0A060C1
:101990003D4808602C493E48086034480068017A98
:1019A0000129D6D1F720E07000F084F83BE038E060
:1019B0002FE026E011E02D480068017A012932D19C
:1019C0000572002001F0ACFB40F28F1000F022FB0A
:1019D000AFF257201C49086025E02F486060E1788D
:1019E000F72902D0EF2906D01DE0204A0121126814
:1019F00051722A4903E01D4909684D722849016165
:101A000011E02848284960600C48086003F0A0FFF6
:101A100009E02648244960600948086003F098FFFF
:101A200001E023486060012000F076FF20786070BC
:101A300070BD00008C0E0020980E002002000020D7
:101A4000060000209D1E000810000020651B0008F5
:101A5000AC0E0020580000204C9A0008C00E002058
:101A6000D40E0020889A00086A7E00080C0000202E
:101A7000E80E0020191D0008C9670008FC0E0020B0
:101A8000100F0020300D002059150008B514000873
:101A9000B51A0008240F0020380F0020509B0008C2
:101AA000489B00084C0F002020000020600F002001
:101AB000740F002010B52248224C01782078F729B5
:101AC00008BF401C03D0EF2908BF401E00D1207082
:101AD00010F0FF0010D0022884BF02202070607830
:101AE000217888421CBF002000F016FF20780128D2
:101AF0001AD002281ED112E0134805F0BFF90020C9
:101B000000F00AFF1148006805F0B8F9012000F064
:101B100003FF10490E480860002020700EE00E48B8
:101B200005F0ACF90D4803E0074805F0A7F90C48AB
:101B3000FFF7D0FD012000F0EFFE2078607010BDAF
:101B40008F0E0020600E0020780E0020940E0020E2
:101B50007D17000810000020640E0020EE0C00200D
:101B6000F00C002070B55B4D5B4C29782078EF2994
:101B700008BF401C03D0F72908BF401E00D12070C9
:101B8000C0B20521FF280CBF2170052807D921709C
:101B9000002001F02BFC52495048086070BD60786D
:101BA000217888421CBF002000F0B6FE207806286D
:101BB00046D2DFE800F003283C515A63494805F05B
:101BC0005DF9494E0020F0722878FD2802D0FE28E9
:101BD00013D079E0A078642838BF0A3074D2A0709E
:101BE000C2B2424906F10800FEF720FB40484149D5
:101BF00000680661A078088066E0A078002818BF19
:101C00000A3861D0EBE73C4805F038F929783B48C1
:101C1000FD2902D0FE2904D056E00188FF2913D304
:101C200052E0018800294FD013E001804CE0344895
:101C300005F024F929783348FD2902D0FE2906D081
:101C400042E00188FF293FD20188491CEDE7018865
:101C5000D1B30188491EE8E72B4805F00FF90020B1
:101C600004F0EEFD03F038FE2EE0284805F006F9FA
:101C7000012004F0E5FD03F02FFE25E0244805F0E7
:101C8000FDF82878234DFD2802D0FE280CD01BE05B
:101C90002878022818D2002000F00CFA012000F069
:101CA00009FA2878401C09E0287868B1002000F083
:101CB00001FA012000F0FEF92878401E2870C0B219
:101CC00004F062FD04F018F9012000F025FE2078F0
:101CD000607070BD8F0E0020600D00207D17000821
:101CE00010000020640D0020DC0D0020FC9900088D
:101CF000900E002034440140780D0020380400404C
:101D00008C0D002034040040A00D0020B40D0020F4
:101D1000C80D0020500000202DE9F0414F4E504CDE
:101D200031782078EF2908BF401C03D0F72908BF7D
:101D3000401E00D12070C0B20421FF280CBF2170CA
:101D4000042808D92170002001F0CEFB46494548FF
:101D50000860BDE8F0816078217888421CBF0020CF
:101D600000F0DAFD2078414F414D052866D2DFE8CA
:101D700000F0030A375058003E4805F07FF8002075
:101D800004F0B8F95AE03C4805F078F83078FD28BE
:101D900002D0FE281DD051E028688179052938BF7E
:101DA000491C4BD2817128683449807900EB80004E
:101DB00001EB40003968086131482061002000F0E3
:101DC000E1FF30482061002000F0DCFF03F0D6FF87
:101DD00034E028688179002918BF491E2ED0E1E738
:101DE000294805F04BF83078FD2802D0FE2807D0AE
:101DF00024E039682548086129680120487105E018
:101E000039682348086129680020487103F0B6FF4B
:101E100014E0204805F032F81948206104F064FC11
:101E20000CE01D4805F02AF828688079042818BFBE
:101E300005280AD0396848F671404881012000F031
:101E40006BFD20786070BDE8F08139684EF6A030F7
:101E500048810C48206104F047FCEFE78F0E00201A
:101E6000E80D00207D17000810000020900E0020D3
:101E70000C000020FC0D0020100E0020009A00082D
:101E8000EA0D0020EE0D0020240E00203C9A0008F0
:101E9000449A0008380E00204C0E002070B54A4DC0
:101EA0004A4C29782078F72908BF401E03D0EF2933
:101EB00008BF401C00D12070C0B20026FF2804BF1C
:101EC0000520207002D0052888BF26706078217810
:101ED00088421CBF002000F01FFD207806286CD22D
:101EE000DFE800F003054B4D4F5339484AE03948CD
:101EF00004F0C4FF2878FB285FD137480680001F14
:101F000006803648008803F0C3FA64230F22AA2112
:101F1000C32002F047FE4FF6FF7003F0BFFA002027
:101F200004F08EFC2E4D2868008803F0B7FA2D4B84
:101F30000022BE21C32003F057F92B4B0022BE2103
:101F400040F2131003F050F900F098FA012004F069
:101F500077FC2868008803F0A1FA244B0022BE21F8
:101F6000C32003F041F9204B0022BE2140F21310A0
:101F700003F03AF900F082FA1FE01D4802E01D4824
:101F800000E01D4804F07AFF17E01C4804F076FFDB
:101F90002878FB2811D1012000F022FC18480068A5
:101FA00004F06CFF012003F073FE17491548086028
:101FB00016490120487016494870012000F0ACFC19
:101FC0002078607070BD00008F0E00208C0F002004
:101FD000900F0020A40F0020380400402E000020A5
:101FE00058000020689B0008549B00085C9B000878
:101FF000B80F0020CC0F0020E00F0020F40F0020CD
:10200000940E00207D170008100000200200002020
:102010000600002010B50446002000F04BF8012017
:1020200000F048F8002001F039FB0A2000F0AAFE79
:1020300019480A21008800F0A9FD18480A210088E3
:1020400000F0A4FD16481849048016480288A0181C
:10205000401CC0F34F0008804AF2D73100FB011347
:10206000190D6FF0180301FB03001049C0B208708E
:10207000801A401E0028B8BF40420870012001F0BD
:102080000DFB0B4800680079002808BF10BD012037
:10209000BDE8104004F02EB8EE0C0020F00C00203B
:1020A00038000020360000203200002051000020BF
:1020B0000C0000202DE9F0411A4D0028D5F80880C9
:1020C0000CBF19481948A860287838B1012808D0F1
:1020D00000F032F8C5F80880BDE8F08100F0CEF8D5
:1020E000F8E7134E134F002430883988401A801EB9
:1020F0000028EFDDA8680119388891F826332044BC
:10210000821C401C92B291F8251380B200F02EF987
:10211000601C84B230883988401A801EA042E9DCF5
:10212000D8E70000500000205C000020A20600203C
:1021300038000020360000202DE9F84F4548DFF830
:1021400018B100260088BBF80010401AB11E01EB40
:10215000400080B2009003F005FE009800240028A3
:1021600070D9DFF8F8A03E4DDFF8F890A868204459
:1021700090F82513BBF800003044401C80B203F0F7
:102180001DF9A868204490F8261390F82503081A32
:102190001FFA80F8A8F10100BE2828BF4FF00108FF
:1021A0000127B8F1000F46D0A868BAF800202044F3
:1021B00090F82513781E0844904247D0BBF80020C1
:1021C0003244531C284A128893423FD0274A82FB4C
:1021D00000325310A3EBE272524202EB820210185B
:1021E0000AD16878224A3044A2FB0032D2086FF04C
:1021F000180302FB030048B3381D08441C49A1FB27
:102200000021C9086FF0180201FB020050B968787C
:1022100018493044A1FB00218908494201EB8101A2
:10222000081813D01448008802F0B2FF3846791C11
:102230008FB24045B8D1701C86B2A01C84B2009801
:10224000844293D3BDE8F84F03F016BDB9F80000FF
:10225000EAE70000380000203600002034000020AB
:1022600050000020300000203200002067666666C3
:102270001F85EB51CDCCCCCC2C0000202DE9F05F9C
:10228000314F324E002438883188401A0028D8BF98
:10229000BDE8F09FDFF8B8A0DFF8B8B0DFF8B8907D
:1022A000DFF8B8802E4DBAF80020A868204490F8D6
:1022B00025030119914244D03188BBF80020214404
:1022C000491C91423DD0A9FB00218908494201EBFC
:1022D000810109180AD16978224A2144A2FB0132FE
:1022E000D2086FF0180302FB031151B31D49401DC2
:1022F000A1FB0021CA086FF0180102FB010048B9D8
:1023000068782044A9FB00218908494201EB81013A
:10231000081816D01448008803F0BAF8A8682044BA
:1023200090F8251330882044401C80B202F026FC2F
:10233000601C84B238883188401AA042B3DCBDE802
:10234000F09FB8F80000E7E73800002036000020D2
:102350003400002032000020CDCCCCCC3000002056
:10236000500000201F85EB512C0000202DE9F84F74
:1023700005460C46181B914698460028B8BF4042B7
:102380000090444534BF4FF0010A4FF0FF3AC0F1CE
:10239000010603F0E7FC0098C0F1000B2F4800880D
:1023A000844227D02E480088854223D02D48A0FBA8
:1023B00004218908494201EB810109190FD12A49F9
:1023C00049786A18294909881144294A091DA2FB3C
:1023D0000132D3086FF0180203FB021151B1244AF5
:1023E000611DA2FB0132D2086FF0180302FB03113A
:1023F000A1B902E01F48078812E01B4949786A1812
:102400001A4909881144091DA0FB01208008404297
:1024100000EB8000401808BF164800D01648078817
:102420002146284602F0CAFF384602F0B1FE4D456B
:1024300008BF44450DD07000584503DD0099761A59
:10244000691C8DB20128A9DA04EB0A00761C84B25B
:10245000A4E7BDE8F84F03F00FBC000034000020F3
:1024600032000020CDCCCCCC500000203600002023
:102470001F85EB51300000202C0000202DE9F04F8B
:10248000664EDFF8A08183B031680020DFF890B19C
:10249000DFF894A1C870A8F1040900BFBAF80000E1
:1024A00002F0F6FF614864230F2201880120CDE984
:1024B0000001AA21C32002F0ABF94EF6A03002F0D1
:1024C000E7FF30680022C07800EB8001584800EB3D
:1024D0004103BE2140F2431002F086FE55A30022C4
:1024E0009621C32002F080FE04F046FA002528461B
:1024F00004F0E0FF4FF06632504B04F03FFE002244
:102500004F4B04F087FD04F091FF80B201230E22AF
:10251000AA2102F041FA3068584507BFA8F80050D8
:10252000B8F80070A9F80050B9F800700A2000F05F
:1025300094F8002404F086F8022818BF002434D050
:10254000681CC5B2FF2DD2D3BAF8000002F0A0FF7C
:102550000025009564230F229621C320019502F0E7
:1025600057F9002C4ED037A300229621C32002F049
:102570003BFE00BF4FF4967000F06FF800956423A7
:102580000F229621C320019502F042F9306800889D
:1025900002F084FF3068C178491CC9B2C1700629B5
:1025A000FFF47CAF03B0BDE8F08F03F0D7FAD6F8A4
:1025B00000C000210CF104009CF805205FF07F03AF
:1025C00010F802EF1444427871445B1EF8D1601891
:1025D0009CF8031100240844C0F307207D38072825
:1025E000AED219489CF803108445184830F81120E1
:1025F00018BF02F47F423A4408BF120220F81120AB
:102600000124A1E74FF4784002F048FF10A3002214
:102610009621C32002F0E8FDACE70000580000203E
:102620005C000020380400402C0000202E00002018
:102630004C9A000857414954000000006666044067
:10264000006068404F4B0000A206002042000020BE
:1026500046616C75726500007047002140F271227E
:102660005043B1EB001F38BF491CFAD3704700003C
:102670002DE9F05F4E4F4F4C4F4D3E8828B34EF63C
:10268000A03002F005FF28880023001F81B2F01E51
:1026900080B20722804602F07FF920880023C01C08
:1026A00081B20722404602F077F9788802F0F0FE06
:1026B000298820880123091A0B398AB2401D81B26A
:1026C0003046BDE8F05F02F067B9DFF8F080B8F897
:1026D000000002F0DDFE28880023001F81B2F01EFA
:1026E00080B20722074602F057F920880023C01C59
:1026F00081B20722384602F04FF92088401D84B28B
:102700002888401F8442A8BFBDE8F09FDFF8B0A032
:10271000DFF8B0B0DFF8B0902C4F00BFBAF800007F
:1027200086421CBFBBF8000084423FD02848018885
:1027300028480078081A321A2748511E80FB0130B9
:102740004310A3EBE070404200EB8000401808D13A
:10275000611DA9FB0130C0086FF0180300FB0310D6
:1027600020B3501E89FB0021CA10A2EBE1716FF06B
:10277000180201FB020040B91848A0FB04108008B1
:10278000404200EB8000001910D0B8F8000000BFF4
:1027900002F07EFE2146304602F0F0F9601C84B261
:1027A0002888401F8442B9DBBDE8F09F3888EFE7F6
:1027B000F20D00203C0000203A0000202C000020F8
:1027C00032000020340000201F85EB513000002033
:1027D000360000205100002067666666CDCCCCCC68
:1027E00010B5040082B04FF0000021D002F050FE7E
:1027F000124901200988CDE90001114801881148DA
:102800000088091A8BB210490A8810490988521A9F
:102810000A3A491D92B289B201F0FAFF022C04BFB4
:1028200002B010BD012002B0BDE8104000F036BF7C
:1028300002B0BDE8104000F031BF00002E000020C3
:1028400038000020360000203A0000203C00002024
:102850002DE9F04707460C4602F052FB8246642FF2
:1028600088BF64278CB94FF6FF7002F011FE042375
:102870000622E02140F26D1002F094F91B230F2292
:10288000DB2140F2711002F08DF9002540F28B1926
:10289000B5EB970F38BFDFF8788018D20024A9EB8A
:1028A000050600BF08EB4400B0F82C0102F0F0FD73
:1028B00004F1DC01B0B289B202F060F9601C84B2AC
:1028C0000E2CEFD3681C85B2B5EB970FE6D31148F9
:1028D000008802F0DDFD01230422E12140F27110A5
:1028E00002F05AF8A9EB9704B4F5B97F0AD3012393
:1028F0000D22DC21204602F04FF8601E84B2B4F5B0
:10290000B97FF4D25046BDE8F04702F0C1BD0000E7
:102910009C7E00082A0000202DE9F043744D0646F5
:10292000002428688BB0002804BF0BB0BDE8F083FA
:102930004FF6FF7002F0B2FD6E4802F057FD6E498F
:102940002868884243D1012E0BD140F6410002F0A5
:102950009FFD28688388C2884188008802F022F998
:1029600001242868008902F093FD4CF6596100208B
:10297000CDE90001286841888388C2880088091B46
:10298000001B89B280B201F043FF4EF6A03002F086
:102990007FFD28680422418883880088091B091D5F
:1029A000001B89B280B202F01DF94FF4B07002F042
:1029B0006FFD28681C234188C2880088091B001B02
:1029C00089B280B202F0EEF80BB0BDE8F083012EC0
:1029D0007ED0B0F808804FF6FF77012428684FEAD0
:1029E000D821C8F34512C08808F01F030DF10C0967
:1029F000002857D0A9F1020C10F0010F14D0C80222
:102A000000EB421018442CF8020F481E1E283CBF51
:102A1000481CC1B2501E3E283CBF501CC2B2581EBA
:102A20001E283CBF581CC3B22868C088400839D053
:102A30004FEAC12808EB42189844ACF80280A1F193
:102A40000108B8F11E0F3CBF491CC9B2A2F1010830
:102A5000B8F13E0F3CBF521CD2B2A3F10108B8F14D
:102A60001E0F3CBF5B1CDBB24FEAC12808EB4218CB
:102A700098442CF8048FA1F10108B8F11E0F3CBF57
:102A8000491CC9B2A2F10108B8F13E0F3CBF521C6B
:102A9000D2B2A3F10108B8F11E0F3CBF5B1CDBB240
:102AA000401EC5D1CDE90076CDF80890286883880E
:102AB000C2884188008801F041FE2868621E418872
:102AC000036911440088E21C104489B280B200E01E
:102AD00005E0012202F088FB0BB0BDE8F083074956
:102AE000B0F80A8080890F8802F0D8FC76E70000F1
:102AF000900E0020EC990008740F00202A0000209E
:102B000030B583B0002003F09BFE124D124C2868B4
:102B10002188038880780091421CCDE90123431D60
:102B2000C01E81B20022104601F0E2FE012003F037
:102B300087FE28682188038880780091421CCDE9AF
:102B40000123431DC01E81B20022104601F0D0FEB9
:102B500003B030BD5800002036000020094900B500
:102B60000968094B83B089781B884A1CCDE900327B
:102B700002904B1DC81E81B20022104601F0B8FE23
:102B800003B000BD58000020360000202DE9F05FA2
:102B90000646801EDFF874815D4F5E4C85B20029C9
:102BA00033D00A297DD04FF4784002F071FC2088A0
:102BB0000023401F81B20522284601F0EDFEB8F83F
:102BC00000000023001D81B20522284601F0E4FE2A
:102BD00048F6714002F05CFCB8F80000801D85B238
:102BE00020880A38A842D8BFBDE8F09F01230422FC
:102BF0002946304601F0D0FE05F10A0085B2208852
:102C00000A38A842F2DCBDE8F09F4348008802F091
:102C10003FFC20880023401F81B20522284601F096
:102C2000BBFEB8F800000023001D81B20522284633
:102C300001F0B2FEB8F80000801D85B22088093886
:102C40008542A8BFBDE8F09FDFF8D0A0DFF8D0B084
:102C5000DFF8D090DFF8D080BAF8000086421CBFC1
:102C6000BBF8000085423DD0304831490078321A27
:102C7000501C81FB00314B10A3EBE171494201EB89
:102C80008101081808D1681DA9FB0031C9086FF03F
:102C9000180301FB030028B3501C89FB0021CA1054
:102CA00000E022E0A2EBE1716FF0180201FB0200EC
:102CB00040B92048A0FB05108008404200EB80008E
:102CC00040190FD0B7F8000002F0E2FB2946304669
:102CD00001F054FF681C85B2208809388542BBDBAF
:102CE000BDE8F09FB8F80000EEE7388802F0D0FBAE
:102CF0002188B8F800000123091A10398AB2801D12
:102D000081B23046BDE8F05F01F046BE3C000020D5
:102D10002C0000203A0000202E000020320000206D
:102D2000340000201F85EB513000002051000020AE
:102D300067666666CDCCCCCC10B504460E4884B030
:102D4000012C01880D48026808BF518812880C4B7D
:102D5000501C80B21B880093CDE90101501D83B245
:102D6000D01E81B20022104601F0C2FD04B0204600
:102D7000BDE8104000F006B82C000020F80D00203F
:102D8000360000202DE9F05F5049514E514D524F11
:102D9000F0B10A287DD048F6714002F079FB308806
:102DA000401C84B22888401EA042D8BFBDE8F09FD6
:102DB0003868002306220188204601F0EDFD04F169
:102DC0000A0084B22888401E8442F1DBBDE8F09FEF
:102DD000288832880024801A401E0028D8BFBDE809
:102DE000F09FDFF8F8A0DFF8F8B0DFF8F890DFF830
:102DF000F8803868BAF800100088884246D03188D8
:102E000021444A1CBBF800108A423FD03749A1FB3D
:102E100000329208524202EB820212180AD1344A5E
:102E200012782244A9FB02C3DB086FF0180C03FBE5
:102E30000C2252B3401DA9FB0032D2086FF01803D8
:102E400002FB030050B92A4800782044A1FB00216E
:102E50008908494201EB8101081817D01B480088F6
:102E600002F016FB3868018830882044401C80B28C
:102E700001F084FE601C84B228883188401A401E0C
:102E8000A042B6DCBDE8F09F03E0FFE7B8F8000021
:102E9000E6E7088802F0FCFA298830880023091A3E
:102EA000491E8AB21349401C80B2098801F074FDA2
:102EB000298830880023091A491E8AB20E49401C0D
:102EC00080B20988BDE8F05F01F066BD2C000020EB
:102ED0003600002038000020F80D002034000020CB
:102EE000320000201F85EB5130000020CDCCCCCC2F
:102EF00051000020EA0D0020EE0D00202DE9F04FDA
:102F0000DFF854A183B0BAF8000001F0AFFF002051
:102F100002F0BEFA5148534C01880120CDE900016E
:102F20004F4801882088091A8BB24F490A884F49B7
:102F30000988521A0A3A491D92B289B201F068FC16
:102F4000012000F0ABFB00F09DF8002003F078FCBE
:102F5000474D21882868038880780091421CCDE97C
:102F60000123431DC01E81B20022104601F0C0FCA7
:102F7000012003F065FC286821880388807800918F
:102F8000421CCDE90123431DC01E81B20022104620
:102F900001F0AEFC642701F0B3FF83464FF6FF70EB
:102FA00002F076FA04230622E02140F26D1001F0CF
:102FB000F9FD1B230F22DB2140F2711001F0F2FD1D
:102FC000DFF8B080002540F28B190024A9EB05063C
:102FD00008EB4400B0F82C0102F05AFA04F1DC01CD
:102FE000B0B289B201F0CAFD601C84B20E2CEFD3DE
:102FF000681C85B2B5EB970FE7D3BAF8000002F072
:1030000047FA01230422E12140F2711001F0C4FCCF
:10301000A9EB9704B4F5B97F0AD301230D22DC2173
:10302000204601F0B9FC601E84B2B4F5B97FF4D239
:10303000584602F02DFA4FF6FF7002F02FFA0E48B4
:1030400002F0D4F903B00122BDE8F04F0BA3DC215C
:103050004FF49B7002F0C8B82A0000202E00002018
:1030600038000020360000203A0000203C000020FC
:10307000580000209C7E0008EC9900084650533A06
:103080000000000010B52548A0F120046060002079
:10309000FFF742FC04F1340060600020FFF73CFCC5
:1030A00004F1480060600020FFF736FC04F15C008A
:1030B00060600020FFF730FC04F1700060600020C9
:1030C000FFF72AFC04F1840060600020FFF724FC75
:1030D00004F1980060600020FFF71EFC04F1AC00D2
:1030E00060600020FFF718FC04F1C0006060002061
:1030F000FFF712FC04F1D40060600020FFF70CFC25
:1031000004F1E80060600020FFF706FC04F10C0009
:103110006060BDE810400120FFF7FEBBAC0E002050
:103120002DE9F0410025904F904EDFF84482914CFC
:1031300082B0002800F090804FF49670FEF76AFF8E
:1031400047F67F6002F0A4F9B8F800102088012348
:10315000091A0B398AB2401D81B2308801F01CFC7B
:10316000854803F08BFE0020FFF7D6FB834803F071
:1031700085FE0020FFF7D0FB4FF6FF7002F08EF9BE
:103180007F4C4B20804A20807E488049804E0068DA
:1031900090427AD1088802F00BF920887DA379301B
:1031A00081B2002240F2311002F01EF820887BA389
:1031B0006B3081B2002240F2311002F015F8208805
:1031C00078A35D3081B2002240F2311002F00CF899
:1031D000208876A34F3081B2002240F2311002F0F5
:1031E00003F8208873A3413081B2002240F23110ED
:1031F00001F0FAFF2580308802F0DAF8208865A314
:10320000793081B2002240F2311001F0EDFF2088C8
:1032100062A36B3081B2002240F2311001F0E4FF72
:10322000208860A35D3081B2002240F2311001F0AD
:10323000DBFF20885DA34F3081B2002240F23110C5
:1032400001F0D2FF20885BA3413081B2002240F21E
:10325000311001F0C9FF7CE0388802F019F90095BF
:1032600001953088B8F80020C0F5C7718BB221886D
:10327000401E521A0C3A891D92B289B280B201F0F6
:10328000C7FA02B0BDE8F081FFE74C4A904260D136
:10329000088802F08DF8208849A3793081B2002295
:1032A00040F2311001F0A0FF208847A36B3081B2BB
:1032B000002240F2311001F097FF208844A35D30D6
:1032C00081B2002240F2311001F08EFF208842A32B
:1032D0004F3081B2002240F2311001F085FF20888A
:1032E0003FA3413081B2002240F2311001F07CFF57
:1032F0002580308802F05CF8208831A3793081B2D3
:10330000002240F2311001F06FFF20882EA36B30B5
:1033100081B2002240F2311001F066FF20882CA318
:103320005D3081B2002240F2311001F05DFF208853
:1033300029A34F3081B2002240F2311001F054FF36
:10334000208827A3413081B2002240F2311001F0E1
:103350004BFF2548006803F091FD388802B0BDE8B6
:10336000F04102F025B800002C00002038000020B9
:103370003A0000203C000020640E0020780E00205F
:10338000EC0C0020300D0020B51400085C0000207B
:10339000A2060020205670703A00000020645420DD
:1033A000203A0000205664633A00000020524D533A
:1033B0003A000000204443253A0000005915000857
:1033C000205620313A000000205620323A000000FA
:1033D0006D61783A000000006D696E3A00000000EF
:1033E000202020463A000000940E002070B5324D97
:1033F000324E334C82B000283DD0022002F048FC0F
:103400004FF49B70FEF706FE47F67F6002F040F82F
:10341000318820880123091A0B398AB2401D81B2F4
:10342000288801F0B9FA2748006803F021FD2648F2
:1034300003F024FD0020FFF76FFA244803F01EFD7F
:103440000020FFF769FA224803F018FD0020FFF77B
:1034500063FA204803F012FD0020FFF75DFA1E48D2
:1034600003F00CFD0020FFF757FA02B01B48BDE83F
:10347000704003F003BD1A48008802F009F80020EC
:103480000090019028883288C0F5C7718BB22188DE
:10349000401E521A0C3A891D92B289B280B201F0D4
:1034A000B7F91048006803F0E9FC02B00120BDE85C
:1034B000704002F0EDBB0000380000203A00002010
:1034C0003C000020900E0020640D0020780D0020AC
:1034D0008C0D0020A00D0020B40D0020C80D002090
:1034E0002C000020940E002070B5304D304E314C31
:1034F00082B000283AD0022002F0CAFB4FF49B7041
:10350000FEF788FD47F67F6001F0C2FF3188208812
:103510000123091A0B398AB2401D81B2288801F0B3
:103520003BFA2548006803F0A3FC244803F0A6FCFE
:103530000020FFF7F1F9224803F0A0FC0020FFF77C
:10354000EBF9204803F09AFC0020FFF7E5F91E484C
:1035500003F094FC0020FFF7DFF91C4803F08EFC19
:1035600002B00020BDE87040FFF7D6B918480088C7
:1035700001F08EFF00200090019028883288C0F56D
:10358000C7718BB22188401E521A0C3A891D92B223
:1035900089B280B201F03CF90E48006803F06EFC7D
:1035A00002B00120BDE8704002F072BB380000207C
:1035B0003A0000203C000020900E0020FC0D00206E
:1035C000240E0020100E0020380E00204C0E00208B
:1035D0002C000020940E002010B5002833D040F2BB
:1035E0008F10FEF717FD0220FFF7FAF81F4800685A
:1035F00003F03EFC1E4803F041FC0020FFF78CF96D
:103600001C4803F03BFC0020FFF786F91A4803F042
:1036100035FC0020FFF780F9184803F02FFC00204C
:10362000FFF77AF9164803F029FC0020FFF774F938
:10363000144803F023FC0020FFF76EF9BDE81040AA
:10364000104803F01BBC0120FFF7CAF80E480068C1
:1036500003F014FC012002F01BFB0D490B4808602D
:103660000C49012048700C49487010BD900E002094
:10367000900F0020A40F0020B80F0020CC0F0020D6
:10368000E00F0020F40F0020940E00207D170008AA
:103690001000002002000020060000202DE9F05F4D
:1036A00000280CBF51485248008801F0F1FE514FEC
:1036B000DFF844A1DFF844B13988BAF800000023EC
:1036C000091A8AB2BBF8001001F066F94C4DDFF818
:1036D0003481DFF834912988B8F800000123091AF1
:1036E0000B398AB2401D81B2B9F8000001F054F9DB
:1036F000B9F800603888864218D200BFB8F80000D8
:10370000401D84B22888401F844209DA2146304691
:1037100001F034FA601D84B22888401F8442F5DB32
:1037200006F1190086B238888642E7D3BAF800005D
:10373000B9F800600A30B0421AD200BFB8F80000F1
:10374000401D84B22888401F844209DA2146304651
:1037500001F014FA601D84B22888401F8442F5DB12
:10376000A6F1190086B2BAF800000A308642E5D800
:10377000BBF80060B8F80000864214D9BAF80040DF
:103780003888844208D23146204601F0F7F9601D9E
:1037900084B238888442F6D3A6F1190086B2B8F80C
:1037A00000008642EAD82888BBF80060401F8642A5
:1037B00015DA00BFBAF800403888844208D2314692
:1037C000204601F0DBF9601D84B238888442F6D3CC
:1037D00006F1190086B22888401F8642EADBBDE860
:1037E000F05F4FF6FF7001F053BE00002C00002088
:1037F0003000002038000020360000203400002077
:103800003A0000203C000020320000202DE9F04763
:103810007D4F0024651E39887C4E30882A0CDFF8E5
:10382000F081DFF8F09100297AD0A1F56E41EE39F0
:1038300038D0A1F58851113905D0384600F08EFBFB
:1038400004286ED1CFE098B1A0F56E41EE3938462C
:1038500016D100F083FB042818BFBDE8F0870021D3
:10386000304600F0A3FB042818BFBDE8F087C7E08E
:10387000384600F073FB042818BFBDE8F087BFE0AE
:1038800000F06CFB042808D10021384600F08EFBC4
:10389000042804BF304600F061FB042818BFBDE8CF
:1038A000F087ADE088B190423CD1304600F056FB45
:1038B000042818BFBDE8F0870021384600F076FBE9
:1038C000042818BFBDE8F0879AE0F98838F814009A
:1038D000814208BF25B2AC420ED04E4900F09EF89E
:1038E000012809D038F81400B9F8001000F0C6F823
:1038F000042818BFBDE8F087601C84B2072CE4D30D
:103900000021384600F052FB042818BFBDE8F087BC
:10391000304600F023FB042818BFBDE8F0876FE0B5
:1039200013E069E0384600F019FB042808D10021B3
:10393000384600F03BFB042804BF304600F00EFB85
:10394000042818BFBDE8F0875AE060B1904218BF64
:10395000DFF8C4A01AD1304600F000FB042818BFDD
:10396000BDE8F0874CE0384600F0F8FA042808D1AA
:103970000021384600F01AFB042804BF304600F04E
:10398000EDFA042818BFBDE8F08739E0BAF8000066
:1039900038F81420904208BF25B2AC420FD01D4920
:1039A000104600F03BF8012809D038F81400B9F8A7
:1039B000001000F063F8042818BFBDE8F087601C11
:1039C00084B2072CE2D30021304600F0EFFA04283D
:1039D00018BFBDE8F087384600F0C0FA042818BFC9
:1039E000BDE8F0870CE00021384600F0DFFA04283B
:1039F00004BF304600F0B2FA042818BFBDE8F087D3
:103A00000420BDE8F087000000F0010800F4010880
:103A1000520D00204E0D002006F4010830B4144D64
:103A2000002201242B88DFF84CC0BCF800C033B161
:103A3000BCF1000F0FBF0122AB2030BC704705EB7B
:103A400082239B1CDFF830C00CEB82229A4207D9FC
:103A5000B2F800C0844506D132F8020C0880002478
:103A6000204630BC7047121F9A42F1D8F8E7000098
:103A700000F0010800F40108FEF3010870B5184BCE
:103A800005460E461A8800201649098801244EF67C
:103A9000EE6CA9B1002A1CBFAB2070BD614500D1FE
:103AA0002046114903EB802401EB8020844205D29B
:103AB0002268521C07D0241DA042F9D8802070BD76
:103AC0006245EED0ECE73146204600F06FFA04285C
:103AD00018BF70BD2946A01CBDE8704000F066BA52
:103AE00000F0010800F40108FEF301082DE9F0419F
:103AF0001B4988701B494FF400330B601A4C9E0120
:103B000026601A4A4FF0007CC2F810C0184F4FF0E0
:103B100011353D603D1DD5F8008060F31F28081F5A
:103B2000C0F800804FF40078C2F810804FF002080F
:103B3000C1F800800B60C2F810C04FF088313960C6
:103B40002968C9B241F47F410160802020600120D2
:103B5000FEF783FD28682660C0F30720BDE8F081EA
:103B600008100020100C0140100801400010014016
:103B7000040C01402DE9F041374E4FF40037376017
:103B80003649B8010860364980000861401230604B
:103B9000344D28684088C043C1B2002000F066F868
:103BA00028684088C043C0F30721012000F05EF878
:103BB00028680088C1B2042000F058F828680088FE
:103BC000010A052000F052F8274C002020702078D0
:103BD00040F00501062000F049F80D20FFF786FFB0
:103BE000A080AE281CBF0120BDE8F0810020FFF7B7
:103BF0007DFFA080FE281BD10120FFF777FFA0806A
:103C0000FF2815D10420FFF771FFA08090280FD165
:103C10000520FFF76BFFA08029680988B0EB112F02
:103C200006D10620FFF762FFA0802178884202D0EB
:103C30000220BDE8F081286800883760C1B2042006
:103C400000F014F828680088010A052000F00EF83A
:103C50000020BDE8F0810000100C01401008014078
:103C6000001001400C000020081000202DE9F00396
:103C70001C4CA0701C4A4FF4003313601B4D4FF4D2
:103C8000000CC5F800C0DFF868C01D02CCF8105069
:103C9000184E4FF011373760371DD7F80090A2F15A
:103CA000040860F31F29C8F800904FF40079CCF89D
:103CB00010904FF00209C2F800901360CCF8105039
:103CC000D7F800C061F31F2CC8F800C0C2F80090FC
:103CD00013604FF044323260062808BF2170BDE8FF
:103CE000F003704708100020100C0140100801403C
:103CF00000100140040C014070B5544C00212046D6
:103D000003F0F2F80821204603F004F9504D012198
:103D1000284603F005F90221284603F007F90A2195
:103D2000204603F0F1F80021284603F0D7F801F00F
:103D3000EDF8002000F0DAFC002001F097F80020F8
:103D400001F036FB4FF4784001F0A8FB41494020D8
:103D50000860414801F04AFB40A30022C8214620E8
:103D600001F042FA0A20FEF778FC434801F03EFBDE
:103D700062B6002002F064FD02F0FEFD012002F0B8
:103D80005FFD02F0F9FD3D490120086072B64FF079
:103D900000014FF4001001F07DFE47F67F6001F056
:103DA0007DFB37A30022A021142001F01DFA0A2078
:103DB000FEF753FCFFF7DEFE012825D002282ED0A7
:103DC00035A300228C21142001F00EFA3AA3002220
:103DD0007821142001F008FA0A20FEF73EFC142195
:103DE0000420FFF743FF02F02DFC002822D001F051
:103DF000B5FE3BA300226421142001F0F5F9BDE8D3
:103E000070406420FEF729BC4FF4784001F046FB77
:103E10003AA300228C21142001F0E6F9FEE74FF4CA
:103E2000784001F03BFB3EA300228C21142001F0DE
:103E3000DBF9FEE74FF4784001F030FB40A30022AD
:103E40006421142001F0D0F9FEE7000000100140C9
:103E50000008014010080140788D0008566572691D
:103E60006669636174696F6E20205065726970685D
:103E70006572616C000000001894000884E100E0A5
:103E8000426F7468204C54433133383020697320BA
:103E90004F4B2E2E2E000000526561642045504D80
:103EA00035373020636F6E74726F6C2072656720D7
:103EB0004F4B2E2E2E00000045504D3537302072CE
:103EC0006561642F777269746520726567697374C0
:103ED000657273206973204F4B2E2E2E0000000058
:103EE0005772697465206379636C65205352414D44
:103EF000206973204F4B2E2E2E0000005265616406
:103F00002045504D35373020636F6E74726F6C20D2
:103F1000726567206572726F722E2E2E000000008F
:103F200045504D353730206572726F722072656171
:103F3000642F7772697465207265672E2E2E0000DB
:103F40004572726F72207772697465206379636C51
:103F500065205352414D2E2E2E00000030B50546EF
:103F60004FF4302000F04AF8042818BF30BD0A4C46
:103F7000206940F0020020616561206940F0400046
:103F800020614FF4302000F039F8216941F6FD72CC
:103F90001140216130BD000000200240024801694B
:103FA00041F08001016170470020024070B5054674
:103FB0000E464FF4005000F021F8042818BF70BDE1
:103FC000074C206940F0010020612E804FF4005022
:103FD00000F014F8216941F6FE721140216170BDB4
:103FE0000020024003480249416003494160704794
:103FF0002301674500200240AB89EFCD174A0146F7
:104000000420D36813F0010F08D0A9B1D3680420AD
:1040100013F0010F18BF01201BD10FE0D36813F07C
:10402000040F18BF022004D1D26812F0100F18BF7D
:104030000320002918BF704705207047D36813F08C
:10404000040F18BF022004D1D36813F0100F18BF5B
:104050000320491E0128D8D0EBE7000000200240D1
:104060002DE9F001CB78002203F00F0C13F0100FB4
:104070001CBF8B7843EA0C0C0B884FF00F0613F033
:10408000FF0F4FF0010518BF046819D00F8805FA1B
:1040900002F31F409F420FD1970006FA07F824EA67
:1040A00008040CFA07F73C43CF78282F08BF436178
:1040B00002D0482F08BF0361521C082AE6D30460CF
:1040C0000A88FF2A87BF44680022BDE8F0017047D4
:1040D00002F108030F8805FA03F31F409F420FD136
:1040E000970006FA07F824EA08040CFA07F73C439D
:1040F000CF78282F08BF4361CF78482F08BF0361CE
:10410000521C082AE4D34460BDE8F0017047000067
:1041100070B5644CA06940F00400A061A06940F053
:104120000800A061A06940F01000A061A06940F003
:104130000100A0615C48416841F400614160416850
:1041400041F00071416059494FF011300860594801
:10415000574A026042140A61574A4A60584A57490E
:104160001160E16941F00101E161C10442F20F72A5
:104170000A854FF47A728A8581220A8001238B8115
:1041800041044FF0E0250023C5F80011DFF834C1E9
:10419000E0218CF80010E16941F00201E161DFF8F3
:1041A00028C11321ACF800100CF1040CFF21ACF86D
:1041B0000010DFF818C17F21ACF800100CF1040CDE
:1041C000ACF800104249B1F800C04CF0680CA1F8FE
:1041D00000C0B1F800C04CF4D04CA1F800C03D497B
:1041E000B1F800C04CF0010CA1F800C0B1F800C05B
:1041F0004CF0100CA1F800C03749B1F800C04CF4E5
:10420000004CA1F800C035490A80354908220A80CF
:10421000CB70FFF725FFA06940F40070A061314822
:10422000016841F001010160016821F46021016031
:10423000016841F4801101602B48016841F460611C
:1042400001602A49032008602948016841F02001E3
:1042500001604FF48020C5F880012649F0200870E5
:10426000A06940F40060A061234948F69F4008809F
:10427000091D4FF4FA60088020498010088020480A
:10428000018841F0600101801E48018841F480717D
:104290000180001F018841F081010180BDE870406C
:1042A00001F0B6BF001002400000014000100140C4
:1042B00011010011000801401100100011109900B7
:1042C000000C01401CE400E02804004034040040DD
:1042D0001804004020040040440400400004004052
:1042E000240000200824014010240140342401400F
:1042F0000424014012E400E0282C0140342C014049
:10430000182C0140042C0140FEE700004FF47840D7
:1043100001F0C4F803A30022A021142000F064FFE0
:10432000FEE700004572726F72207768656E20614B
:104330006363657373696E67204C5443313338305F
:1043400000000000838A0022008B43EA004020F036
:104350007F4031EA000008BF012210467047002963
:10436000018814BF41F0010121F001010180704773
:104370000029018814BF41F4807121F4807101800B
:1043800070470029018814BF41F4007121F40071C5
:104390000180704700220B0F21F07F4112BF1430C3
:1043A000090C18300068084218BF012210467047F7
:1043B00070B50446808886B00D4620F03F066846FA
:1043C00001F074FB29490298B0FBF1F189B246EA89
:1043D0000102A280228822F001022280244B2A6856
:1043E0009A4209D85200B0FBF2F080B2042838BFDC
:1043F0000420491C218424E0EB88A3F53F4CBCF148
:10440000FF0C05D102EB4202B0FBF2F080B208E0F3
:1044100002EBC20303EB0212B0FBF2F080B240F4F5
:1044200080400205120D08BF40F0010040F400403A
:104430004FF4967251434FF47A72B1FBF2F1491C7A
:104440002184A083208840F0010020802088A98852
:104450006A8920F00A0020F480601143084320801C
:10446000A88929890843208106B070BD40420F0009
:10447000A0860100002A14BF41F0010101F0FE01F5
:1044800001827047018270472DE9F05F364D374A4F
:10449000374EA8681288817890F82633891AC91F88
:1044A0008FB290F825133088821C401C92B280B2E3
:1044B000FDF75CFFA8684179394480F8251300882E
:1044C00000F0E6FFDFF8AC8031880124B8F8000086
:1044D000401A801E0128D8BFBDE8F09FDFF898B0D1
:1044E000DFF89890DFF898A0DBF80000407A012808
:1044F0000DD1A8680119308891F826332044821C18
:10450000401C92B291F8251380B2FDF72FFFA868E6
:10451000204441793944C9B280F82513B9F8002004
:10452000921F914204DCBAF80020921D914201D200
:1045300080F82523318890F8253304EB010C0CF129
:1045400001018AB290F824131FFA8CF000F0D0FA1F
:10455000601C84B2B8F800103088081A801EA0428F
:10456000C2DCBDE8F09F00005000002034000020B5
:1045700036000020380000200C0000203A00002007
:104580003C0000202DE9F05F4C4DDFF83491A86825
:10459000B9F8001082780088511AC91F1FFA81F8F3
:1045A00000F076FF474F484E002438883188401A83
:1045B000801E0028C6BFDFF81491DFF814A1BDE803
:1045C000F09F44480068407A01284DD101F0CAFBB1
:1045D000A868204490F8251339480088814227D0E4
:1045E00030882044421C3C480088824220D03B4B0B
:1045F000A3FB01208008404200EB800040180BD153
:104600006878374A2044A2FB00C24FEAD20C6FF010
:1046100018020CFB020058B131484A1DA0FB02C031
:104620004FEAD00C6FF0180000FB0C2080B903E0BB
:104630002C48B0F800B00EE068782044A3FB0032AC
:104640009208524202EB8202101808BF254800D09F
:104650002548B0F800B030882044401C80B200F0FB
:10466000ADFE584600F094FDA868204441794144CD
:10467000CAB280F82523B9F80010891F8A42C8BF42
:1046800080F8251390F82523BAF80010891D8A4276
:1046900038BF80F8251390F8251330882044401C3B
:1046A00080B200F06BFA601C84B238883188401AFE
:1046B000801EA04285DCBDE8F09F00005000002075
:1046C0003400002038000020360000203A0000208E
:1046D0003C0000200C00002032000020CDCCCCCCCF
:1046E0001F85EB51300000202C00002070B5114CCC
:1046F0000125A188226805FA01F1090411610E4E15
:1047000010B15A2807D00BE01C21162001F00AFB3B
:104710000020307004E0BC21162001F003FB35704E
:10472000A088216805FA00F00861BDE8704000F03B
:1047300063BE000048100020141000202DE9F04F47
:1047400083B005460E461746DDE90C102F4ADDF80A
:1047500038909A461180591C1FFA81FB691E8CB251
:104760000091711E1FFA81F8019110B101280DD03E
:1047700022E001233A464146204600F00DF900238D
:104780005A464146204600F007F915E005EB0A00BD
:10479000791C401E8AB280B20123414600F0FCF829
:1047A000F019401E81B200235A46204600F0F4F86A
:1047B000009885B2019886B201F0D4FAAA44AA45BD
:1047C00084BFDFF84880374419D93146284600F0C5
:1047D000F5FD3446A7420ED909EB4400A0EB460094
:1047E0000088A8F80000B8F8000000F0D1FC601CB8
:1047F00084B2A742F0D8681C85B2AA45E5D801F07A
:104800003BFA03B0BDE8F04F00F0F6BD1A100020EF
:104810002DE9F84F044635480A9F0E46B0F800903F
:1048200090461D46008801EB080A04EB050B00903A
:104830001FFA8AF31FFA8BF13246204600F066FE1B
:104840002A490B980880681C631E711E08F101023A
:10485000012F06D085B29CB2022F21D0032F2DD07C
:104860003CE09CB28DB296B287B201233246294613
:10487000204600F091F8E01980B201233246294623
:1048800000F08AF800233A462946204600F084F8D2
:10489000A81981B200233A46204600F07DF81DE0B9
:1048A00089B2012342460E46204600F075F80023E7
:1048B0002A463146204600F06FF80FE00BF1010068
:1048C00080B2012392B2314600F066F80AF101008D
:1048D00081B200232A46204600F05EF80348A0F883
:1048E0000090BDE8F84F00F087BD00001A100020CE
:1048F0002DE9F04186B062F30F04DDE90D76DDF8B5
:10490000308060F30F0C68F30F0563F31F4467F307
:104910001F45CDE9005461F31F4CCDF808C0BDF828
:104920000A40BDF806C01A4A02AB01A869466445B0
:1049300023D2BDF80250AC4224BF1160C2E901305D
:1049400006D2AC4534BFC2E90101C2E901101360CF
:104950001068516892680F4B0068096812681E80E1
:1049600014460D46064600F045F806B02246294694
:104970003046BDE8F04100F0F3B9BDF80240936065
:10498000A44534BFC2E90001C2E90010E0E700001D
:10499000501000201A1000202DE9F04105460F4666
:1049A0001446984601F0DEF93946284600F006FD27
:1049B0000F4EB8F1010F11D0308800F0E9FB284606
:1049C000691C8DB2394600F0F9FC2100A4F1010008
:1049D00084B2F1D1BDE8F04101F04EB9308800F069
:1049E000D7FB2000A4F101018CB2F7D1F2E700005F
:1049F0001A1000202DE9F04F044605468BB21FFA2D
:104A000080FCA3EB0C0085B00028B8BF40420FFA31
:104A100080F84FEA114BABEB144000B200909C457C
:104A200034BF01204FF0FF300190009891B2A8EB05
:104A3000000006B2ABB2C81A0028B8BF40420FFA55
:104A400080F9100CA0EB15400FFA80FA8B4234BFAE
:104A500001204FF0FF300290A9EB0A0007B2009846
:104A600040420390CAF100000490200C584504BF56
:104A700005B0BDE8F08F71000AB203998A4206DDE5
:104A80000099711A0EB20199214461F30F04424555
:104A900005DA06EB0801401C0EB260F31F447800F3
:104AA00001B20498814206DDA7EB0A0007B2029822
:104AB000284460F30F05494506DA07EB090007B201
:104AC000280C401C60F31F451FFA84FCA8B28445E3
:104AD00006D2A0EB0C0082B2210C0023604604E059
:104AE000ACEB00018AB2210C0023FFF755FFBCE7B5
:104AF0002DE9F04F0746D41B83B00E4690469946E9
:104B0000002CB8BF6442A9EB06000028B8BF4042A1
:104B10000090474534BF01204FF0FF3001904E45D3
:104B200034BF4FF0010A4FF0FF3A0098251A01F008
:104B300019F90098C0F1000B3146384600F03EFCF0
:104B40000D48008800F024FB474508BF4E450ED0B5
:104B50006800584504DD00996D1A019939448FB2F7
:104B6000A042E9DA06EB0A00254486B2E4E703B086
:104B7000BDE8F04F01F080B81A10002070B504466F
:104B80000D4601F0EFF82946204600F017FC0448D6
:104B9000008800F0FDFABDE8704001F06DB800003B
:104BA0001A1000202DE9F0411C4605460E46174616
:104BB0000123FFF7F1FE281980B201233A4631465E
:104BC000FFF7EAFE0023224631462846FFF7E4FEBF
:104BD000F01981B222462846BDE8F0410023FFF7D4
:104BE000DBBE00002DE9FF4F8DB0002000900F9834
:104BF000181A01900028DCBF11B0BDE8F08FDDE984
:104C00000E100844059080B2411A03914942069162
:104C10000E99081A0890404207900D990098084490
:104C20000A90DDE90E5186B208441FFA80F90B9014
:104C30000598A9EB060480B20490002CB8BF64422A
:104C400003980028B8BF069802904E4534BF012053
:104C50004FF0FF3009900498854234BF4FF0010AAD
:104C60004FF0FF3A0298271A01F07CF80298DFF81B
:104C7000EC80C0F1000B2946304600F09FFBB8F8ED
:104C8000000000F085FA4E4504BF049885420ED01E
:104C90007800584504DD02997F1A099931448EB293
:104CA000A042E8DA05EB0A00274485B2E3E700F00A
:104CB000E3FF0B980F9985B20598DDF838A087B20D
:104CC0000A9800EB41001FFA80F9A9EB0504002CBB
:104CD000B8BF644208980028B8BF079802904D45B5
:104CE00034BF01204FF0FF300490574534BF4FF0E0
:104CF000010B4FF0FF3B0298261A01F033F802989F
:104D0000C0F100083946284600F058FB13480088D7
:104D100000F03EFA4D4508BF57450ED070004045A3
:104D200004DD0299761A049929448DB2A042E9DA89
:104D300007EB0B00264487B2E4E700F09DFF0099E3
:104D40000F9801EB400080B20090DDE90001814244
:104D50003FF763AF11B0BDE8F08F00001A100020DC
:104D60002DE9F04F144615461FFA81FC93B2ACEBC7
:104D7000030287B0002AB8BF52420FFA82F84FEA06
:104D8000114ACAEB14410FFA81F9634534BF01217E
:104D90004FF0FF3101914FF0FF310391A8EB090172
:104DA0000EB282B2ABB2D11A0029B8BF49420FFA93
:104DB00081FB290CA1EB104000B20090934234BF5C
:104DC00001204FF0FF3002904FF0FF300490009828
:104DD000ABEB000007B2C9F100000590009840421B
:104DE0000690210C514504BF07B0BDE8F08F70005C
:104DF000059A00B2904206DDA6EB090216B2019AAE
:104E0000224462F30F04404506DA06EB080006B2BE
:104E10000398084460F31F447800069900B2884262
:104E200006DD0099791A0FB20299294461F30F0542
:104E3000584507DA07EB0B0007B2049800EB154062
:104E400060F31F45A0B21FFA85FC604505D2ACEBAC
:104E500000018AB2210C002305E0A0EB0C0082B215
:104E6000210C00236046FFF797FDBAE72DE9F04FCC
:104E70000546002400F0C0FA1B4801228188D0F8C2
:104E800000B002FA01FA4FEA0A41CBF810101A48B2
:104E90001649174BB0F804C0164FDFF860E002FA6D
:104EA0000CFC1B88006809684FEA152805F0FF090B
:104EB0004FEA0C428D6837F818601D403543CD60CD
:104EC0000261C0F810C08D6837F819601D40354385
:104ED000CD600261C0F810C0641C7445EAD1CBF803
:104EE00010A0BDE8F08F0000481000202410002022
:104EF00020100020729B0008401000200077010065
:104F00000148C088704700001410002030B59A484E
:104F100001248188006804FA01F1016197488188C1
:104F2000006804FA01F1016195488188006804FA7B
:104F300001F1016193488188036804FA01F21104C8
:104F40001961012140F2712C002001FB0CF100BF1E
:104F5000B0EB011F38BF401CFAD31A6105210020B5
:104F600040F27122514300BFB0EB011F38BF401C1B
:104F7000FAD3854DA888296804FA00F00004086176
:104F80000221832000F0CEFE0321852000F0CAFE1E
:104F900093218C2000F0C6FE0121912000F0C2FE7A
:104FA0000021832000F0BEFEB0213E2000F0BAFEBA
:104FB00003213F2000F0B6FE1021402000F0B2FE99
:104FC0005621412000F0AEFE1321422000F0AAFE3F
:104FD0004621432000F0A6FE2321442000F0A2FE3B
:104FE0007621452000F09EFE4F21462000F09AFEDB
:104FF0005F21472000F096FE4F21482000F092FEEE
:105000004F21492000F08EFE6121172000F08AFE1A
:10501000F9212B2000F086FE0A21002040F27122A7
:10502000514300BFB0EB011F38BF401CFAD314211D
:105030001B2000F077FE11211A2000F073FE0D21D5
:105040001C2000F06FFE3D211F2000F06BFE14219C
:10505000002040F271225143B0EB011F38BF401CC9
:10506000FAD30A21192000F05DFE1A21192000F060
:1050700059FE2821002040F271225143B0EB011F5C
:1050800038BF401CFAD31221192000F04BFE282112
:10509000002040F271225143B0EB011F38BF401C89
:1050A000FAD320211E2000F03DFE3221002040F2E4
:1050B00071225143B0EB011F38BF401CFAD360216D
:1050C0003C2000F02FFE40213D2000F02BFE382137
:1050D000342000F027FE3821352000F023FE38214F
:1050E000242000F01FFE2821002040F271225143AD
:1050F000B0EB011F38BF401CFAD33C21242000F044
:1051000011FE1C21162000F00DFE0621012000F0EA
:1051100009FE0021552000F005FE0021022000F0CC
:1051200001FE0021032000F0FDFD0021042000F01D
:10513000F9FDEF21052000F0F5FD0021062000F02B
:10514000F1FD0021072000F0EDFD0121082000F015
:10515000E9FD8F21092000F0E5FD222000F0A4F9EF
:105160000A4840F28F110181EF214181A888296806
:1051700004FA00F0086130BD30100020401000201B
:1051800038100020281000204810002014100020A3
:1051900070B4114909688B68104A114CB2F800C00C
:1051A00003EA0C02030A34F813301A43CA600D4AAA
:1051B000012395881268AB401D04156113618E6848
:1051C000C0B206EA0C0C34F810004CEA0000C860CB
:1051D0001561136170BC704724100020201000205E
:1051E000729B0008401000202DE9FF4F6D488DB0E4
:1051F0000168002919BF10990029002011B008BFCB
:10520000BDE8F08F0978002900F0C7800D9805905F
:105210000E980290DDE90FA00278624800920068C3
:10522000017842788368C1EBC201CDB28178009ADF
:10523000A2EB010C022202EB8C029A5AC368802472
:1052400002EB030930B1009A564F914202D8C1785F
:105250008A4202D94FF0000864E000F083FD00208C
:1052600001903868827881680098801A31F82000AF
:10527000002888BFC5F1080B49D901990598084451
:10528000099080B2029900F099F83868029E4FF0B8
:105290000008407800282CD95FF0000599F800003C
:1052A000204204D040480088FFF772FF08E0BAF1BE
:1052B000000F3AD00998711C80B289B200F07EF8D4
:1052C000701C86B2386864084078401E404508BFAC
:1052D000AB4503D0681CC5B2082DDFD308F101002F
:1052E00000F0FF083868802409F101094078404542
:1052F000D2D80198401CC0B2019038688278816889
:105300000098801A31F8201001988142B5D800F039
:10531000B3FC3868827881680098801A31F82000E0
:1053200000F0FF080F9828B128E020480088FFF718
:105330002FFFC5E700F016FD1A4E002530680079F2
:10534000002819D90D98194F00EB080909EB050041
:1053500080B20E9900F032F800243888FFF718FF69
:10536000601CC4B230680078A042F6D2681CC5B296
:1053700030680079A842E9D800F07EFC094800684E
:1053800001790D984044084480B20D901098401C5B
:105390001090007800287FF439AF0D9811B0BDE867
:1053A000F08F0000101000201610002018100020B0
:1053B00001498880704700001410002030B5044671
:1053C0000D46090A022000F0ADFCE9B2032000F00E
:1053D000A9FC210A062000F0A5FCE1B2072000F09C
:1053E000A1FCBDE83040222000F05EB80149086011
:1053F0007047000010100020F0B523480024254617
:10540000037840F28F11EF2213B1012B06D00AE08E
:1054100040F28F14EF250181428104E0EF2440F235
:105420008F1502814181194E0127B088316807FA32
:1054300000F0000408610021022000F073FC00214C
:10544000032000F06FFC290A042000F06BFCE9B295
:10545000052000F067FC0021062000F063FC00211D
:10546000072000F05FFC210A082000F05BFCE1B29D
:10547000092000F057FC222000F016F8B0883168AF
:1054800007FA00F00861F0BD141000204810002059
:105490000149C8807047000014100020014948806D
:1054A0007047000014100020134A30B49188012383
:1054B000126803FA01F14FEA014CC2F810C0DFF89C
:1054C0003CC0DCF800C0DCF808400D4D2D882C40B5
:1054D0000C4D35F810002043CCF80C00DFF828C044
:1054E000BCF8040003FA00F0DCF8003004041C618E
:1054F0001861116130BC7047381000202410002062
:1055000020100020729B0008401000202DE9F04F71
:10551000DFF8EC8005460F46B8F804004FF0010AAA
:10552000D8F800100AFA00F00004DDF824901646BE
:105530001C460861110A022000F0F4FBF1B20320BE
:1055400000F0F0FB210A042000F0ECFBE1B20520A2
:1055500000F0E8FB290A062000F0E4FBE9B207208E
:1055600000F0E0FB390A082000F0DCFBF9B209206A
:1055700000F0D8FB2220FFF797FFB8F80400D8F816
:1055800000800AFA00FBC8F810B0781B401CA11B71
:10559000491C00FB01F24FEA0B40C8F810001C4800
:1055A0001849194CB0F804C0184B0AFA0CF52488B5
:1055B000006809684FEA192609F0FF074FEA054C11
:1055C000D1F8089033F816A009EA040949EA0A0953
:1055D000C1F80C90C0F810C00561D1F8089033F8FC
:1055E00017A009EA040949EA0A09C1F80C90C0F8B1
:1055F00010C00561521EE3D2C8F810B0BDE8F08FAC
:10560000481000202410002020100020729B000869
:10561000401000202DE9F0410121284801F0AAFBAB
:105620002648274C274D0088274B010AA170C2B29B
:10563000AA7018880A388142C8BFA07007DCB3F886
:1056400002C00CF10A0C614538BF84F802C08242E6
:1056500003DC58880A30824200D2A87006211B4819
:1056600001F088FB002001F0EBF8194F174E1949A3
:105670003868C07836F81000000A0880012001F070
:10568000DFF838681449C07836F81000C0B20880D6
:1056900004F5497005F549714FF4C872A378437059
:1056A000AB784B70A37800F8023FAB7801F8023F6B
:1056B000521EF3D1BDE8F04100F01EBC3E000020B8
:1056C0005C000020A20600203A00002042000020DA
:1056D0005800002038040040340400402DE9F84F01
:1056E0006F48704F704D00883988DFF8C091401ABC
:1056F0006FF0010101EB400080B20090A868B9F89A
:105700000020002681780088891AC91F4FFA81FB82
:10571000FFF7BEFE0098002400288CBFDFF890A1A0
:10572000BDE8F88F63480068407A012869D100F02D
:1057300019FBA868204490F825135A480088304483
:10574000401C80B2FFF73AFEA868204490F8261368
:1057500090F82503081A1FFA80F8A8F10100BE2866
:1057600028BF4FF001080127B8F1000F47D0A86803
:10577000B9F80020204490F82513781E0844904280
:105780007DD0484A12883244531C4B4A12889342B7
:1057900075D04A4A82FB00325310A3EBE2725242A8
:1057A00002EB820210180BD16878454A3044A2FB04
:1057B0000032D2086FF0180302FB030000286BD000
:1057C000381D08443E49A1FB0021C9086FF01802AA
:1057D00001FB020050B968783A493044A1FB00212E
:1057E0008908494201EB8101081855D036480088E4
:1057F000FFF7CEFC3846791C8FB24045B7D100F098
:105800003BFAA868204441795944CBB280F825334B
:105810008179594401F0FF0C2C4980F826C30A888D
:10582000921F9342C8BF80F8252390F82573284A19
:1058300013889B1D9F4238BF80F825330988891F34
:105840008C45C8BF80F8261390F826331188891D2F
:105850008B4238BF80F8261390F8262390F8251342
:10586000501A82B2501EBE2828BF01220D480123C3
:1058700000883044401C521E80B292B200E00BE01F
:10588000FFF78AF8701C86B2A01C84B2009884428C
:10589000FFF448AFBDE8F88FBAF80000A8E70000B1
:1058A0003800002036000020500000203400002086
:1058B000300000200C000020320000206766666681
:1058C0001F85EB51CDCCCCCC2C0000203A00002021
:1058D0003C000020FEE7704770B517480078FD28AF
:1058E00008BF012504D0FE280CBF4FF0FF3570BD66
:1058F000124C13492068098880780A31884217D9E8
:10590000104909880A39884212DA0F480088FDF7E1
:1059100025F90E4801784A1C027020680A2981780E
:1059200026BF05EB850211442944817000F026FA58
:10593000BDE87040FDF7E4B88F0E0020580000204D
:105940003C0000203A0000202A000020890F00209F
:1059500070B51F4D1F4CE9782068F72916D0EF2944
:1059600018BF70BD8178002914BF491E70BD8170B9
:1059700011F0FF0F1CBF012141700DD020681649A6
:105980008278012A0ED0022A13D018E081780229E9
:1059900038BF491CEBD370BD002141700078FCF783
:1059A00089FBEBE7C078097881430620FEF75EF9B2
:1059B00005E0C078097801430620FEF757F9206812
:1059C0000649807801EB80006968086170BD0000BD
:1059D0008C0E002020000020081000203C9B0008B6
:1059E0007047000070B51148114DA0F10C04A06083
:1059F0002868007A012809D1A078411CA1700A28E2
:105A000004D90C48006880470020A0702868407ABC
:105A1000012806D100F016FE022818BF70BD00F064
:105A20009DF86068BDE87040004700005C00002001
:105A30000C000020300D002070B51248124DA0F26D
:105A40005264A0602868007A012809D1E078411CDE
:105A5000E1700A2804D90D48006880470020E070F2
:105A60000B48407850B92868407A012806D100F0E8
:105A7000E9FD022818BF70BD00F070F86068BDE84D
:105A800070400047A20600200C000020300D0020CE
:105A900002000020044A0029D16914BF084321EA0A
:105AA0000000D061704700000010024026494A689B
:105AB00012F00C03254A18BF042B01D0082B01D08B
:105AC000026015E04A684B6802F470124FF0020C55
:105AD00013F4803F0CEB924203D04B6813F4003F69
:105AE00003D01B4B5A43026002E0184B5A4302603A
:105AF0004A68184B02F0F00212099A5CD0F800C014
:105B00002CFA02F24260D1F804C00CF4E06C4FEAC7
:105B10001C2C13F80CC022FA0CFCC0F808C0D1F8F9
:105B200004C00CF4605C4FEADC2C13F80C30DA4053
:105B3000C2604968084B01F44041890B595CB2FBD3
:105B4000F1F10161704700000010024000127A007C
:105B500000093D003D0D0020390D00202DE9F05FCA
:105B60003A4EDFF8EC803088B8F80010401A394916
:105B70000978484387B20F20FDF7B8FF36494FF048
:105B8000883008600D1D2868291DC0B240F47F4090
:105B9000086032488024046031494215DFF8C4C0EF
:105BA00009684305C97901291FD12F49B8F8008038
:105BB00036880988A1EB0808711A884515DDA8EB1D
:105BC00001010E04360CA6F1010189B20DD000BF0F
:105BD000CCF81020CCF81030CCF81020CCF81030D5
:105BE0000E00A1F1010189B2F2D1791E89B24FF400
:105BF000000647B31F4FDFF87480DFF874B097F8E2
:105C0000009000BFCCF8102004602F684FEA172ADC
:105C100008EB010787F805A00660CCF81030046097
:105C20002F680BEB010A3F0A8AF805700660B9F18C
:105C3000020F1CBFCCF81020CCF810300F00A1F1DF
:105C4000010189B2DED10660BDE8F09F3800002076
:105C5000360000204E000020040C014010080140D6
:105C60000C00002000100140F20D00205C0000201C
:105C7000A20600205000002003480122818800680D
:105C800002FA01F1016170474810002070470000DE
:105C900010B51449144C01280FD0022818BF10BDAC
:105CA0002068007A0870012818BF10BD0020FDF799
:105CB00037FA21680020087210BD0878012805D045
:105CC000BDE8104040F28F10FCF7A4B94FF4967075
:105CD000FCF7A0F90120FDF723FA216801200872E2
:105CE00010BD0000340D00200C00002001490861A7
:105CF00070470000E80D002010B5094C206840886E
:105D0000C043401EC1B20020FDF7B0FF20684088AC
:105D1000BDE81040C043C0F307210120FDF7A6BF36
:105D20000C00002010B50C46FFF7BEFB09480068C8
:105D30008168094A12881140084A32F81420114338
:105D4000C160074801218288006891400A0402610D
:105D5000016110BD2410002020100020729B00085B
:105D600040100020044801228188006802FA01F1F5
:105D70000904016170470000481000202DE9F04738
:105D8000DFF860910025564CD9F80000564F00F11D
:105D9000060A40792E46A846B0B1544C387840F0F7
:105DA00002010620FDF762FF9AF80000504990B109
:105DB00001281CD0022825D0032830D04D4A0428C1
:105DC00039D005284BD05FE0387820F0020106205A
:105DD000FDF74CFFE8E720780988401AC0F1800001
:105DE0000028B8BF4042C01FC6B2FF254CE0207853
:105DF0000988401AC0F180000028B8BF4042C01F87
:105E0000C5B241E020780988401AC0F1800000281E
:105E1000B8BF4042C01FC5B24FF0010834E020783F
:105E20000988401AC0F180000028B8BF4042C01F56
:105E3000C6B2FF2526E023780888181AC0F1800032
:105E40000028B8BF4042C01FC5B21088181AC0F160
:105E500080000028B8BF4042C01FC6B214E02378BB
:105E60000888181AC0F180000028B8BF4042C01F3F
:105E7000C5B21088181AC0F180000028B8BF40428F
:105E8000C01FC6B24FF00108D9F80000C079012840
:105E9000387818D040F001010620FDF7E7FE00BF7A
:105EA0003878B8F1000F14D040F008010620FDF753
:105EB000DDFE29460220FDF7D9FE3146BDE8F04758
:105EC0000320FDF7D3BE20F001010620FDF7CEFE32
:105ED000E6E720F008010620FDF7C8FEE9E700002C
:105EE0005E0000200C00002008100020A406002006
:105EF000EA0D0020EE0D002010B5094C094A20687B
:105F00000088C1B24FF4003010600420FDF7AEFEEF
:105F100020680088BDE81040010A0520FDF7A6BEF4
:105F20000C000020100C014070B5134C0546208871
:105F3000FFF73EFA1148FFF759FA2088FFF7AEFA4B
:105F40000F4B0122DC214FF4AA70FFF74DF92A46CE
:105F50000CA10B48FAF76AF94FF6FF70FFF79EFAAB
:105F6000074B0122DC214FF4AA70FFF73DF90649E7
:105F70000020087070BD00002C000020EC99000883
:105F8000350D0020256864000000002070470000E7
:105F90003149086840F00100086048682F4A104005
:105FA0004860086820F4102020F0807008600868BD
:105FB00020F480200860486820F4FE0048604FF418
:105FC0001F0088600A68002042F480320A600A6874
:105FD00000F1010012F4003F02D1B0F5A06FF6D13C
:105FE000086810F4003F31D01D48026842F01002EA
:105FF0000260026822F003020260026842F00202BC
:1060000002604868486048684860486840F48060BA
:106010004860486820F47C104860486840F4E81004
:106020004860086840F080700860086810F0007FE1
:10603000FBD0486820F003004860486840F0020048
:106040004860486800F00C000828FAD105494FF074
:106050000060086070470000001002400000FFF878
:106060000020024008ED00E070B51C4805784FF0B4
:106070008040018A21F0010101820720FDF736FDF1
:106080001749194A174C08700021FF28507818D07A
:106090000123DFF858C0012806D0237053709CF804
:1060A0000000022814D009E01078461C167003285E
:1060B0000ED923709CF80000022809D08CF800103B
:1060C00006E0012804D12170094851701170017057
:1060D0002846BDE87040FDF709BD00000A10002009
:1060E0008F0E0020880F00202800002009100020BB
:1060F000890F002070B52449002591F800C023497C
:106100000B785A1CD2B2BCF1FD0F2ED0BCF1FE0FA1
:1061100031D0002808BF70BD0020FCF7A9FA1C4C44
:106120001C4E2088284480B2208031881A4D0A39BC
:10613000884203DC29880A31884200D2218001206C
:10614000FCF796FA154800680179002908BF70BD70
:10615000228829883388511A9A1A9142CCBF01802B
:106160000280BDE87040FFF7C7BE0A700A2B2CBF43
:1061700005250125D0E70A700A2B2CBF6FF0040516
:106180004FF0FF35C8E700008F0E0020890F002078
:10619000F20D002038000020360000200C00002006
:1061A00010B5154C20680079A0B11448FFF79EFD8A
:1061B0000120FCF7E7FD20688079042818BF052836
:1061C00005D10F48FFF792FD0120FCF7DBFD012010
:1061D000FCF74EFA2068007A012818BF10BD012193
:1061E00008480088FCF7D2FC074801210088BDE878
:1061F0001040FCF7CBBC00000C000020EA0D002092
:10620000EE0D0020EE0C0020F00C0020FEE7000058
:1062100070B501214805FFF73DFC1B48C0210180F6
:10622000032181701C21C17001461848FDF718FF39
:1062300017480021012481804BF6FF71C180048141
:10624000A10241810901818142F210710160114D69
:1062500021462846FEF783F80D492846FEF7A8F8A0
:10626000281D018841F4807101800B4D4FF40031ED
:106270002846FEF78FF80028F8D10848046008493E
:106280004FF0D000087070BD24000020000C0140C9
:106290005C100020005400400058004004E100E081
:1062A00020E400E030B52F4C83B00020A0702E48D1
:1062B000E2880188501A2289401E521A80B2911E2B
:1062C000884221DC294909680144091D101A10F08F
:1062D000010F04D14A78002A88BFA270491C401ED1
:1062E000C0F34F02002A18BFA0780DD04B7883422C
:1062F00088BF18468B78834288BF1846891C521E77
:106300001204120CF2D1A070A07880380028B8BF17
:10631000404201F037FC00F0D9FB1549C86101F09B
:106320003DFBCDE90001154D2378627811A105F1FF
:106330000A00F9F77BFFA08805F10A035D3081B2FE
:10634000002240F25910FEF74FFFA088EB1E03B069
:1063500000225D30BDE8304081B24FF4BE70FEF7E0
:1063600043BF0000E80C0020360000205800002049
:106370006C10002025302A2E2A660A00F60C002018
:1063800030B52F4C83B0FF20E0702E48E2880188A2
:10639000501A2289401E521A80B2911E884221DC76
:1063A000294909680144091D101A10F0010F04D190
:1063B0004A78FF2A38BFE270491C401EC0F34F02E2
:1063C000002A18BFE0780DD04B78834238BF1846BA
:1063D0008B78834238BF1846891C521E1204120C57
:1063E000F2D1E070E07880380028B8BF404201F078
:1063F000C9FB00F06BFB1549086201F0CFFACDE94B
:106400000001154D2378627811A105F10F00F9F70D
:106410000DFFA08805F10F034F3081B2002240F23A
:106420005910FEF7E1FEA088EB1E03B000224F30AA
:10643000BDE8304081B24FF4BE70FEF7D5BE00001B
:10644000E80C002036000020580000206C100020CE
:1064500025302A2E2A660A00F60C002030B5374C6B
:10646000374A0020E3881288B4F808C09B1A5B1EE4
:10647000ACEB020CFF219BB2ACF1020283B0934261
:106480002DDC304AACEB030C12681A44121D1CF0D0
:10649000010F07D15378002B88BF1846FF2B38BF58
:1064A0001946521CACF10103C3F34F0CBCF1000FB1
:1064B00015D05378834288BF18468B4238BF19469F
:1064C0009378834288BF18468B4238BF1946921C86
:1064D000ACF101031FFA83FCBCF1000FE9D1A070FD
:1064E000401AE1700028B8BF404201F04BFB00F0B9
:1064F000EDFA1549086001F051FACDE90001154D9A
:106500002378627811A105F11900F9F78FFEA088B0
:1065100005F11903793081B2002240F25910FEF7DB
:1065200063FEA088EB1E03B000227930BDE8304046
:1065300081B24FF4BE70FEF757BE0000E80C002099
:1065400036000020580000206C10002025302A2E34
:106550002A660A00F60C0020F0B5334C33480021BF
:10656000E28800882389161A721E1D1A92B2A81E8C
:1065700083B0824229DC2E4800681044001DAA1A0C
:1065800012F0010F07D110F8011F4FF4804CA1F554
:10659000807301FB03C10023521EC2F34F029AB164
:1065A00090F801C001F58041ACF580770CFB071134
:1065B00010F802CF03F58043ACF58077521E0CFB38
:1065C00007331204120CEBD11944A81BB1FBF0F0F5
:1065D00000F070FF00F0B0FC00F0EAFC00F076FA8A
:1065E0001449C86001F0DAF9CDE90001144D2378AF
:1065F000627811A105F12800F9F718FEA08805F1CD
:1066000028034F3081B2002240F25910FEF7ECFD12
:10661000A088EB1E03B00022BDE8F0404F3081B2ED
:106620004FF4BE70FEF7E0BDE80C002036000020FD
:10663000580000206C10002025302A2E2A660A00FF
:10664000F60C002070B5174C01266670207840F0DB
:1066500080010620FDF70AFB134D08202860012069
:10666000FBF7FBFF2E600E20FDF740FA01281CBF50
:1066700060780028F7D16078002808BF70BD4FF41B
:1066800000710A4801610904016148122860C000D4
:106690002860207820F080010620FDF7E7FA02202C
:1066A000607070BD08100020100C01400010014007
:1066B000490050EAC12018BF04204A0D18BF40F01D
:1066C000010040F2FF72B2EB515F08BF40F00200E0
:1066D000012808BF052070470146012030390A29EA
:1066E00000D300207047000070B52048204D214C99
:1066F0000078FD282CD0FE2818BF70BD0020FCF7C4
:106700001BFB2878411C29700A28206901882CBFAE
:10671000491F491E01801848216900880A880A30EB
:10672000824204D3154800880A38824200DD08807E
:10673000FFF724FB124820610120FCF7FDFA114805
:1067400020610120FCF7F8FABDE87040FCF7D8B9E9
:106750000020FCF7F1FA2878411C29700A282069EA
:1067600001882CBF491D491CD4E700008F0E002072
:10677000890F0020E80D00203C0000203A00002096
:10678000EA0D0020EE0D00200A490B4A012348B112
:1067900001280BD0022818BF704708484860022023
:1067A000107070470648486013707047054848608D
:1067B00013707047500000204E000020DD56000886
:1067C000854500088944000810B50020FFF792FCB9
:1067D0001548811E086115490A78F72A10D0EF2A5A
:1067E00018D0FB2A18BF10BD4EF6A030104909681A
:1067F00048810120FCF790F80F490E48086010BD51
:106800000088012814BFFD2010BD0870BDE81040AD
:10681000FFF76ABF094A00881288521C904288BF5D
:10682000FE20F2D810BD0000EA0D00208F0E0020DF
:10683000900E00207D170008100000203C00002072
:10684000034900280CBF03480348886070470000D4
:10685000500000205C000020A206002070B53C4DD6
:106860003C4CE9782068F7291ED0EF2918BF70BD8D
:106870000179002914BF491E70BD0171C9B2364AA1
:1068800001EB810102EB41026968354B01260A6187
:10689000324AC5E90121136146721046814209D18D
:1068A0000120FCF739F80AE00179022938BF491CB8
:1068B000E3D370BD0020FCF72FF8A868686020685B
:1068C000284D007900B3287820F004010620FDF758
:1068D000CDF92068C671FFF751FA0120FFF70AFCD5
:1068E0002148FFF703FA0120FCF726FA2068807997
:1068F00004281CBF052870BD1C48FFF7F7F9BDE848
:1069000070400120FCF718BA1748FFF7EFF9002094
:10691000FCF738FA1548FFF7E9F90020FCF732FADE
:106920000020FBF7A5FE287840F004010620FDF7C3
:106930009DF9206800210F4AC1710D49128809880C
:10694000891A0180FFF71AFABDE87040FFF7D4BA40
:106950008C0E00200C0000201E9B0008380F002029
:10696000509B000808100020EA0D0020EE0D0020CA
:10697000380000203600002070B501214805FFF7DF
:1069800089F80A20FBF769FE1A4C01212046FDF721
:10699000EFFC194D20462946FDF7D4FC0028F9D01C
:1069A000164D0022286801792046FDF763FD144E3C
:1069B00020463146FDF7C6FC0028F9D02868C0788B
:1069C0000830C1B22046FDF75DFD0E4D2046294638
:1069D000FDF7B8FC0028F9D001212046FDF7D1FCD5
:1069E0000A20FBF73AFEBDE8704000214FF400108A
:1069F000FFF750B800540040010003005800002089
:106A000082000700840007002DE9F05FDFF8A8B0DE
:106A10002A4C4FF0000A05460F464FF001094FF08F
:106A2000040804F10A0652465B4600F057FD4FF099
:106A300000020BD85B462846394600F09FFB05460E
:106A40004D20707002200F46207028E0DFF870B0F3
:106A500028465B46394600F041FD4FF0000213D84E
:106A60005B462846394600F089FB05466B2070706E
:106A70000F460022134B284600F030FD8CBF84F8EF
:106A8000009084F800A00AE00F4B2846394600F039
:106A900075FB0546202070700F4684F8009084F83E
:106AA00001804820B07086F803A028463946BDE82A
:106AB000F05F00F07DBA000000408F40E80C00203D
:106AC00080842E410088C34065CDCD412DE9F0473B
:106AD00004462048204A0068C078105C01F06AF83B
:106AE000214601F07BF8022101F07FF91B4A1D4D80
:106AF00002271B4900264FF020094FF00108A5F19D
:106B00000A04904202D8184A904207DD00F078FF4C
:106B100085F8019084F80080677016E0134A90426F
:106B200002D8134A904207DD00F06AFF85F8019011
:106B3000277084F8018008E06D2169700D49267086
:106B400088428CBF0321042161705621A970EE7028
:106B5000BDE8F08758000020887E0008003C1CC675
:106B600000007A44F20C0020003C1C4600C079C4AE
:106B700000C079440000C6C2F0B5314C314883B042
:106B800021890088E288091A101A081A00F0FAFF11
:106B900005462D480068408801F00CF8294601F0B0
:106BA0001DF82A4901F01AF829490427002504F1A3
:106BB0000A06884202D82749884207DD264900F0A4
:106BC0001FFF6D2171702570677011E023498842A5
:106BD00002D82349884207DD224900F011FF7521C0
:106BE00071702570677003E06E2171702570677099
:106BF0005321B1701C49F570486000F0CFFE2B4660
:106C0000CDE900011A4D6278184905F11E00F9F727
:106C10000DFBA08805F11E036B3081B2002240F20B
:106C20005910FEF7E1FAA088731C03B00022BDE8FA
:106C3000F0406B3081B24FF4BE70FEF7D5BA000061
:106C4000E80C0020360000200C0000200000A041CD
:106C5000F02374C9F02374490024744900C079C436
:106C600000C0794400007A446C100020947E000833
:106C7000F60C0020F0B5364D36490024EA88098824
:106C80002B89521A521E5B1A92B2991E83B020466B
:106C90008A421EDC304995F803C0096811449A1AEB
:106CA000491DAB78521E92B203EB0C0391F800C061
:106CB000BCEB530F3CBF401C80B284BF04F1010CFD
:106CC0001FFA8CF401F10101A2F101021204120C6D
:106CD000ECD154EA000104BF03B0F0BD1F4E002CFC
:106CE00004BF0020306110D0002808BF1C480BD022
:106CF00000F060FF0746204600F05CFF394600F0D8
:106D00007FFE184900F06AFF306100F047FECDE9D0
:106D10000001164C00230422134904F12D00F9F759
:106D200085FAA88804F12D03413081B2002240F297
:106D30005910FEF759FAA88803B00022BDE8F040C8
:106D4000413081B20A4B4FF4BE70FEF74DBA0000DD
:106D5000E80C002036000020580000206C100020B5
:106D60000000C84200004842947E0008F60C002053
:106D7000907E00082DE9F04106460D4672B6FDF7FB
:106D800031F9FCF743FD0D4C002020702078A8421B
:106D900038BF0B4F0DD2207806EB4001207837F832
:106DA0001000FCF73BFE2078401C20702078A842A1
:106DB000F1D3BDE8F041FDF7F1B80000500D00201F
:106DC000520D00202548A0F11404E06072B6FFF7D0
:106DD000DFF8FDF79DF9FCF78FFFFEF71BFCFCF7D2
:106DE0008DF81F484FF480210025016062B6DFF85E
:106DF0007480DFF8749008F104071C4EFFF7D0F997
:106E000098F801000128787804D0012808BFFEF71F
:106E100013FE08E0012802D0FEF7E4FD03E0FEF7D0
:106E2000E1FDFEF709FEE0680079022801BF99F84C
:106E300000000228002000F027F83078012802D155
:106E40002069804735706078401CC0B2607021783E
:106E50000129D3D1FFF768F86570CFE7140000204F
:106E600000E100E00200002009100020880F00204F
:106E700001498860704700008C0E0020014948607D
:106E8000704700008C0E002010B50F4C0F4A04F123
:106E9000AC0361680028C4E9013112680CBF0C48DA
:106EA0000C4818610CBF0020012050720A48814232
:106EB00004D1BDE810400120FBF72EBD0020FBF7F8
:106EC0002BFDA068606010BD8C0E00200C0000201F
:106ED000489B0008509B0008380F0020014A1060B2
:106EE0009180704748100020064A1060101F00294A
:106EF00008BF4FF47F4103D001290CBFFF21704729
:106F00000180704724100020014A10609180704772
:106F100030100020014A1060918070472810002036
:106F2000014A10609180704738100020014A1060BB
:106F300091807047401000202DE9F04106460F4631
:106F400000F05CFB0D46040018BF0120284320F030
:106F50000040C0F17F6010F1E0400FD5002E14BF5B
:106F600001200020384320F00040C0F17F6000F194
:106F7000E0400028A4BF0120F9F7B2FA20462946D4
:106F8000BDE8F08110B500290AD00878002807D0A4
:106F900005487844F9F75CFE002801D0002010BDB8
:106FA0000248784410BD0000962F00008E2F00008C
:106FB00021F00042A2F16052B2F5801F01F00043BF
:106FC00028BFD2F17F6C0BD95FEA001C43EAC202F2
:106FD00042EB507018BF704728BF20F00100704787
:106FE000B2F5801FBCBF184670474FEA410C1CF534
:106FF000001F02D2084600F0BFBE70B500F0AAFA2A
:1070000000000089FFF7F6BF4FF00040A0F58000B8
:107010007047000010B591EA030F48BF83F00043AA
:1070200000F1DA83841A71EB030C05D2121943EBD9
:107030000C03001B61EB0C01DFF824E14FEA115453
:10704000A4EB135C1EEA430F18BF9EEA445F73D0A3
:1070500023EA0E03DCF1200E21EA045143F48013ED
:1070600032D322FA0CFE10EB0E0023FA0CFE41EB99
:107070000E01CCF1200E03FA0EFE10EB0E0051F1C2
:107080000001B1F5801FCCF1200E32D201EB04518A
:1070900012FA0EF2BDE8104058BF7047401C38BFCE
:1070A0005FEA420218BF7047002814BF20F00100B9
:1070B00041F100014FEA410313F5001F38BF70474B
:1070C000A1F1C04100F094BA012A43EB0302ACF1F4
:1070D000200CDCF11F0E32BF4FF0000E23FA0CF330
:1070E00010EB030041EB0451B4EB115FD0D0A1EBE6
:1070F000045101F5801149085FEA300001EB0451A9
:107100000ED350F1000038BF12FA0EFE08D1BDE8D0
:107110001040C9E7401C38BF5FEA4202CAD1C3E74A
:10712000BDE810404FEA410313F5001F38BF704718
:10713000A1F1C04100F05CBA9EEA445F08D011EAB8
:107140005E0FBDE8104004BF01F000410020704711
:10715000BDE8104070B500F0FDF900BF64FBBE3E15
:107160000000E0FF491058BFC1F140415B1058BF1B
:10717000C3F140438B42EFF3008070472DE9C041DB
:1071800030B4DFF8A0C23CEA111418BF3CEA131473
:1071900000F0EC8081EA03051CEA111444EAD5747E
:1071A00018BF1CEA131500F0C780A4EB05044FF0CC
:1071B000004545EAC12145EAC32341EA505143EA6B
:1071C000525304F17F74994204F500344FEAC02011
:1071D0004FEAC22208BF904200F09C804FEA13653C
:1071E0000FF24016765D4FEA134506FB05F7C7F12F
:1071F000807706FB07F74FEAD737A7FB036876428D
:10720000C8F58038A7FB06CE38BFA8F1010807FBF8
:1072100008E64FF0000EA6FB028CE6FB03CEDCF185
:10722000000CCEF1004E38BFAEF1010EA6FB0C589B
:107230004FF000074FF00005E6FB0E87A1FB08C6E4
:10724000A0FB07CE16EB0E0645F10005E1FB076536
:1072500015F1E04E7EBFA4F580345FEA46066D412D
:1072600016F1800745F100054FEA17274FEA066639
:1072700047EA0567A6F1DE46B6F1805F4FEA1525BD
:107280001FD9384624F0010C05EBC471BCF1FE6F28
:1072900001EB0C1102D8F0BCBDE8008124425CBFB8
:1072A00001F5801E9EEAC47F02D4F0BCBDE80081D7
:1072B000244238D4F0BCA1F1C041BDE8004100F047
:1072C00097B94FEAD22242EA43524FEAD323A7FBAF
:1072D00002864FEAD02040EA415007FB03661EEACF
:1072E0000E0F4FEAD12105FB026658BFA6EB0056F0
:1072F000B6EB00564FEA520E4EEAC37E18EB0E0E66
:1073000056EB530EBDD518EB02085E417F1C55F1BC
:107310000005B6E74FF480154FF000074FF0000668
:107320004FF00008ADE7F0BC4FF0000001F1C041A4
:1073300001F00041BDE8008111EA0C1F0CEA1315B1
:1073400000D00CE013EA0C1F00F025804FF0000085
:10735000F0BC81EA030101F00041BDE80081F0BC0E
:10736000BDE8004181EA030100F042B9F0BCBDE88C
:10737000004170B500F0EEF8097EFC3E00F007B861
:1073800081EA03014FF0000001F00041704781EAFB
:10739000030100F02DB9F0BCBDE800414FF0000042
:1073A00021497047FFFDFBF9F7F5F4F2F0EEEDEB44
:1073B000E9E8E6E4E3E1E0DEDDDBDAD8D7D5D4D3F3
:1073C000D1D0CFCDCCCBCAC8C7C6C5C4C2C1C0BF3F
:1073D000BEBDBCBBBAB9B8B7B6B5B4B3B2B1B0AF45
:1073E000AEADACABAAA9A8A8A7A6A5A4A3A3A2A129
:1073F000A09F9F9E9D9C9C9B9A99999897979695E4
:1074000095949393929191908F8F8E8E8D8C8C8B7F
:107410008B8A898988888787868585848483838207
:10742000828181800000FF070000F87F4FEA11533E
:10743000A3F58063D3F11E03A8BFD3F1200C08DBB2
:107440004FF0004242EAC12252EA505232FA03F0AF
:10745000704709420BD4102BC4BF0020704703F5BE
:10746000787CBCF1FF3F05D04FF0FF3070474FF004
:107470000000704770B500F06DF800BF499224809D
:1074800000207047F0E710F0004248BF4042B0FAD9
:1074900080F310FA03F10AD0C3F11D0303F58063F2
:1074A0004FEA415002EB035202EBD12170474FF0FB
:1074B00000007047B0FA80F310FA03F10AD0C3F16C
:1074C0001D0303F580634FEA41504FEA035202EB7C
:1074D000D12170474FF000007047000051EA030CC3
:1074E00017D41CF5801F58BFBCF5801F00F1068023
:1074F000994218BF704708BF9042704707D711F5EF
:10750000801F58BF13F5801F19D4994270478942D4
:1075100070471CF5801F08D5BCF5801FF7D58B423E
:1075200018BF704708BF824270474FF4001C1CEB25
:10753000410F38BF1CEB430F01D28B42704770B52F
:1075400000F008F8922449004FF000514FF08053AA
:10755000FFF708BE0EF1020E2EF0030E5EF8046B6C
:10756000364205D4012A43EB030515F5001F12D856
:10757000012841EB010C1CF5001F0CD80ED14FEA7D
:10758000D17C15F5001F0CEB4C0C0CF1020C08BF64
:107590004CEBD37C04E04FF0080C01E04FEAD37CC5
:1075A0000CEB4C0526FA05F606F00706B6F1040CBE
:1075B00006D20EEB860CBDE870404CF0010C604723
:1075C000DFE80CF0090B02024FF000414FF0000021
:1075D000A1F5002170BD19461046012851EB0104A8
:1075E00018BFD4F5001484BF002001F0004170BD25
:1075F0000808A0F500114FEA310170472DE9F0416C
:1076000001F5801CBCF5001FC0F2C3804FEA115C7D
:1076100021EA0C510CF1FD0C41F480115FEA5C0C85
:107620000CF5C07C01D3400049413DA4890241EAE8
:10763000905187028E0E0A0CA45D04FB04F602FB37
:1076400006F6C6F14046A4FB0662F60D46EA42265F
:1076500006FB06F4A4FB01235242C3F1404338BFAA
:107660005B1EA6FB02420024E6FB0324D20B42EA87
:107670004446A6FB0623A1FB02E2A3FB07E4A418F1
:107680004FF0000252F10002E3FB01426442C2F1FA
:10769000404E38BFAEF1010EA6FB04234FF00002AE
:1076A000E6FB0E32A2FB03464FF00004B61954F17C
:1076B0000004E2FB0264A1FB06E6A4FB07E816EB6C
:1076C00008064FF0000858F10008E4FB0168764214
:1076D000C8F1405838BFA8F10108A2FB06E4A3FB9B
:1076E00008E52D194FF0000454F10004E2FB0854A2
:1076F000A1FB05E6A7FB04E818EB06084FF000061F
:1077000056F10006E1FB048618F1200556F100064B
:10771000A809A8F11B08B10908F03F08B8F10A0F41
:1077200040EA86601CD901EB0C51BDE8F08100BF36
:10773000FCF5EEE8E2DDD8D3CFCBC7C3C0BDB9B608
:10774000B4B1AEACA9A7A5A3A19F9D9B9A9896950D
:107750009392908F8D8C8B89888786858483828194
:10776000A0FB006800FB01F208EB4208B8EB872899
:1077700007D5341858EB0104D5D5401C51F1000150
:10778000D1E7341A78EB0104CDD4401E71F1000129
:10779000C9E75FEA4C0C5FEA9C5C0DD105D34FF062
:1077A000000001F00041BDE8F081BDE8F04170B596
:1077B000FFF7D0FE6DDBFFBEBDE8F0414FF00000EB
:1077C000004970470000F87F10B591EA030F48BFE9
:1077D00083F000433FF526AC841A71EB030C07D20B
:1077E00012198CF0004C43EB0C03001B61EB0C01F5
:1077F000DFF8A4E14FEA1154A4EB135C1EEA430F37
:1078000018BF9EEA445F00F0B08023EA6E03524244
:1078100021EA0451C3EB6E0338BF5B1EDCF1200E7E
:1078200025D322FA0CFE10EB0E0043FA0CFE41EBBE
:107830000E01CCF1200E03FA0EFE10EB0E0051F1FA
:107840000001CCF1200E29D412FA0EF201EB045102
:10785000BDE8104058BF7047401C1CBFB2F1004F3C
:10786000704700280CBF491C20F00100704712EB44
:10787000020E43EB030218BF4FF0010E4EEA420224
:10788000ACF1200CDCF11E0E54D943FA0CFE10EBC7
:107890000E0051F1FF31CCF11E0ED5D50EF1010EC7
:1078A00012FA0EFE404141EB010101EB445C5FEA3C
:1078B0005C5C10D910EBDE7001EB045138BFBEF1F7
:1078C000004FBDE8104018BF704700280CBF491C8E
:1078D00020F00100704730D24FEAD42C11F500118E
:1078E00024F400641BD0B1FA81F20B3AA41AA41E4E
:1078F000D2F12003914030FA03F31943904001EB99
:10790000CC71002C01EB0451BDE81040A8BF7047BA
:1079100001F1C0414FF0000001F000417047B0FAA2
:1079200080F310FA03F100D110BDE41A173C4805AA
:10793000C90AE4E701EB045110BD491001EB045101
:10794000BDE810404FEA300002E04FF00001704700
:107950004A0008BF0042F8D0B2F5001F28BF7047A8
:1079600001F000414FF0000070479EEA445F07D0ED
:1079700011EA5E0FBDE8104004BF002100207047EF
:10798000BDE8104070B5FFF7E5FD00BF40DFF63EF3
:1079900083F00041104670470000E0FF43004FEACB
:1079A000D30C4FEA3C0C43401FBF40070CF1605121
:1079B00013F0FE4F70471CF0006F03D100200CF055
:1079C000004170470CF0004343EA507010B540EAA4
:1079D000CC0000F084F900BF000000924FEA0001E3
:1079E000FFF706BE4FF000414FF00000A1F5002167
:1079F00070470000014800F0C6B900BF0000C07F1A
:107A00004FF47F0C1CEAD0121EBF1CEAD11392EA7D
:107A10000C0F93EA0C0F00F0858090EA010F48BF2D
:107A200042F4807240F4000C41F400002CF07F41DD
:107A300020F07F4000B58142A2EB03020FF2081C48
:107A4000ACEB504EC0F100009EF800E04FEA4E0E45
:107A500000FB0EFC38BF49004FEA2C1C02F5FA026D
:107A60000CFB0EF34FEACE1E4FEA112C4FEAC12158
:107A70000EEB635E42EB22420EFB0CFC4FEA1C5302
:107A800000FB03114FEA112C4FEA01310EFB0CFCF5
:107A90004FEADC4C00FB0C11C14228BF09184CEB2B
:107AA00003335DF804EB10EB410143EBC250B2F538
:107AB0007C0F38BF704729D512F0F00F1CBF00F1C2
:107AC000C04000F000407047008182838485868733
:107AD00088898B8C8D8E8F919293959697999A9C8D
:107AE0009D9FA0A2A3A5A7A8AAACAEB0B2B3B5B7FC
:107AF000B9BCBEC0C2C5C7C9CCCED1D4D7D9DCDFD2
:107B0000E2E6E9ECF0F3F7FAFE0000004FEA400C81
:107B10000CF1807CBCF17E4F28BF7047B0F1C040B3
:107B200000F02AB990EA010F0CEAD11348BF42F4E1
:107B30008072624538BF634507D213F47F0F16D0B9
:107B400080EA010000F00040704710B500F0C7F86F
:107B5000097EFC3E00F005B880EA010000F000401C
:107B6000704780EA010000F0004000F005B912F40F
:107B70007F0F04BF0248704780EA010000F0FCB8A4
:107B80000000C07F10F0004148BF4042B0FA80F3CF
:107B900010FA03F2C3F19D030BD051EAC35101EB7C
:107BA0001220530638BF704700F1010008BF20F0D3
:107BB00001007047B0FA80F310FA03F2C3F19D039D
:107BC0000AD0D90501EB1220530638BF704700F1E7
:107BD000010008BF20F00100704700004FF47F0C47
:107BE0001CEAD0121EBF1CEAD11392EA0C0F93EAD2
:107BF0000C0F00F0478090EA010F48BF42F48072FA
:107C00004FF0004C4CEA00204CEA012102EB030249
:107C1000A0FB0113A2F50002002918BF43F00103E5
:107C20005B0028BF4FEA330342EB22425FEA132C8A
:107C30004CEBC2502EBFBCEB436FB2F57C0F7047CC
:107C40004FEA036CBCF1004F08BF20F00100B2F511
:107C50007C0F38BF70470BD582F0FF0212F5803FD2
:107C6000C8BF704700F1C040D8BF00F00040704767
:107C700000F5000C5FEA4C0C48BF7047B0F1C04003
:107C800000F07AB890EA010F0CEAD11348BF42F431
:107C90008072624538BF634504D280EA010000F07B
:107CA0000040704710B500F01AF800BF8900013E8F
:107CB00000F007B800F009B85FEA410C5FEA1C6CFD
:107CC00008D080EA010000F057B85FEA400C5FEA94
:107CD0001C6CF6D14FF00040A0F5800070470EF10B
:107CE000020E2EF0030E5EF8044B244204D44FEA39
:107CF0004102B2F17F4F11D84FEA4003B3F17F4FF9
:107D00000CD80ED14FEAD07CB2F17F4F0CEB4C0C6B
:107D10000CF1020C08BF4CEBD17C04E04FF0080CD6
:107D200001E04FEAD17C0CEB4C0324FA03F404F09D
:107D30000704B4F1040C06D20EEB840CBDE810402D
:107D40004CF0010C6047DFE80CF0070802024FF02E
:107D50000040A0F5800010BD0846420018BFD2F1D7
:107D6000807288BF00F0004010BD10B5F8F7B0FF7A
:107D70004FF00001016010BDFF2141EAD050C00565
:107D80007047F8F7E4BC0CF00F03092B08BF08207C
:107D900000F053800A2B0BD0082B18BF704708BF88
:107DA0001CF0400F0AD04FF000004FF00001704768
:107DB0001CF0400F18BF4FF0004070471CF0100F30
:107DC00008D020F0704300F07F4242EAD3014FEA2E
:107DD0004370704700F0604021F07F4242EA0002A9
:107DE00001F07F4040EA727070474FF0FF0212EAE4
:107DF000D0521CBF92F0FF038B42C2BFD14200EBB6
:107E0000C1507047002A0AD0002B0BD0002900F087
:107E10000040A4BF40F0FE4040F40000704700F076
:107E20000040704743024FF00B0C18BF4CF0806CC1
:107E30007FF4E0ADAFF3008070471CF4801F11D0D9
:107E40001CF4E02F03D06FEACC31490070474FF0AB
:107E50004050EFF3008222F0704242EA000282F3C7
:107E6000008870474FF000007047010002000400D6
:107E70000A00140028006400C8009001E803D0073D
:107E8000A00F1027204E409C0102050A143200006A
:107E90002500000025302A2E2A660A0001F800F885
:107EA00060F880F8C0F8E0F820F940F980F9A0F90E
:107EB000E0F900FA40FA60FAA0FAC0FA00FB20FBF1
:107EC00060FB80FBC0FBE0FB20FC40FC80FCA0FCD6
:107ED000E0FC00FD40FD60FDA0FDC0FD00FE20FEB9
:107EE00060FE80FEC0FEE0FE20FF40FF80FFA0FF9E
:107EF000E0FFE0FFE0FFE0F7E0EFE0E7E0E7E0DFF2
:107F0000E0D7E0CFE0CFE0C7E0BFE0B7E0B7E0AF59
:107F1000E0A7E09FE09FE097E08FE087E087E07FC9
:107F2000E077E06FE06FE067E05FE057E057E04F39
:107F3000E047E03FE03FE037E02FE027E027E01FA9
:107F4000E017E00FE00FE007E007E007E107E207D6
:107F5000E307E307E407E507E607E607E707E807BF
:107F6000E907E907EA07EB07EC07EC07ED07EE077F
:107F7000EF07EF07F007F107F207F207F307F4073F
:107F8000F507F507F607F707F807F807F907FA07FF
:107F9000FB07FB07FC07FD07FE07FE07FF07FF07C0
:107FA000DF079F077F073F071F07DF06BF067F0624
:107FB0005F061F06FF05BF059F055F053F05FF0420
:107FC000DF049F047F043F041F04DF03BF037F031C
:107FD0005F031F03FF02BF029F025F023F02FF0118
:107FE000DF019F017F013F011F01DF00BF007F0014
:107FF0005F001F001F001F001F081F101F181F1801
:108000001F201F281F301F301F381F401F481F48C8
:108010001F501F581F601F601F681F701F781F7838
:108020001F801F881F901F901F981FA01FA81FA8A8
:108030001FB01FB81FC01FC01FC81FD01FD81FD818
:108040001FE01FE81FF01FF01FF81FF81FF81EF8B1
:108050001DF81CF81CF81BF81AF819F819F818F88C
:1080600017F816F816F815F814F813F813F812F8AC
:1080700011F810F810F80FF80EF80DF80DF80CF8CC
:108080000BF80AF80AF809F808F807F807F806F8EC
:1080900005F804F8000000000000000000000000E7
:1080A0000000071F00077F00071F000003F000000B
:1080B000000000000003F00060000462000763009D
:1080C00003E30000FF00006F800663F007E3300069
:1080D000FB00007F000063E00063700023100003DA
:1080E00000033E00077F000663000663000663008E
:1080F0003FFFC03FFFC0066300066300066B00073A
:10810000E70003C600001E00003300042100062122
:1081100000033300019E000040000020000010001A
:1081200003CC00066600042300042100066000035F
:10813000C00003800007C00007C000066000066E94
:1081400000063F00063F00063B0006F30003E70081
:1081500003C70003860007C00007C00006600004D4
:1081600040000003F001F8000FFF000E07000801B7
:10817000000801000E07000FFF0001F800000400D6
:10818000002C00007800000F00007800004C000078
:10819000040000200000200000200000200000203B
:1081A0000007FF0000200000200000200000200049
:1081B0000020002700001F00000F0000003000001A
:1081C00030000030000030000030000700000700E1
:1081D000000700000800000E000003800000E0001F
:1081E00000380000070000010003FE0007FF000642
:1081F000030006030006030006030006030006034F
:108200000006030006030007FF0007FE000002004F
:1082100000030007FF0007FF00060000070F00072C
:108220008F0007830006C30006E3000663000673A1
:1082300000063300061F00078F00030000070F0031
:10824000070F00060300060300066300066300062E
:10825000630006630006630007FF0007DF0001807C
:108260000001C00001E00001B000019800019C0085
:10827000018C0001860001830007FF0007FF000159
:108280008000018000018000023C00063F000633B0
:1082900000063300063300063300063300063300C1
:1082A00006330007730003E00001C00003F000077D
:1082B000FC00063E00063600063600063300063394
:1082C0000006330006330006320007F40003E00026
:1082D000000F00000F000003000403000603000766
:1082E000030007C30001E300007B00003F00000F14
:1082F0000000070007CF0007FF0006330006330029
:10830000063300063300063300063300063300064A
:10831000330007FF0007CF00003E00027F00066326
:108320000006630006630006630006630003630043
:1083300003630003E30001FF00007E00071C000749
:108340001C00071C00271C001F1C000F1C00001035
:1083500000003800002800006C00006C00004400A1
:1083600000C60000820001830001830001010003B8
:108370000180004400004400004400004400004428
:108380000000440000440000440000440000440099
:10839000004400004400030180010100018300014A
:1083A000830000820000C600004400006C00006CE6
:1083B0000000280000380000100000060000070040
:1083C000000300070300076300077300003B000081
:1083D0001F00000E0001F8000306000401800800E1
:1083E000C010004011F02023F820230C10220610AA
:1083F00022021021021021821023FC10323E1012A2
:10840000022013002009004000C180003E0004004B
:108410000007000007800003E00001F80001BE0033
:10842000018F00018700019F0001FE0001F8000399
:10843000E00007800007000004000007FF0007FFBE
:108440000007FF0006330006330006330006330042
:1084500006330006330007FF0007FF0003CE0003CA
:10846000FE0007FF0007FF000603000603000603E7
:1084700000060300060300060300078F00078F00B5
:10848000038E0007FF0007FF0007FF00060300063A
:1084900003000603000603000603000603000707A7
:1084A0000003FE0001FE0000F80007FF0007FF00C8
:1084B00007FF0006330006330006330006330006CC
:1084C000330006030006030006030006030007FF4F
:1084D0000007FF0007FF0000630000630000630067
:1084E00000630000630000030000030000030003BA
:1084F000FE0007FF0007FF00060300060300060357
:108500000006030006630006630006630007EF0031
:1085100007EF0003E60007FF0007FF0007FF00006A
:10852000300000300000300000300000300000302B
:108530000000300007FF0007FF0007FF0007FF00F3
:1085400007FF0007FF0003C00007C00007C00006C8
:10855000000006000006000006000007FF0007FFFD
:108560000003FF0007FF0007FF0007FF0000700087
:1085700000780000F80001DC00018E00038600078F
:10858000030006030006010004010004000007FFC9
:108590000007FF0007FF00060000060000060000BD
:1085A00006000006000006000006000006000007A6
:1085B000FF0007FF0007FF00000E00003C0000F076
:1085C0000001C00003C00000E000003000000C000B
:1085D00007FE0007FF0007FF0007FF0007FF000777
:1085E000FE00000C0000180000380000700000E0E1
:1085F0000000C00001800003FF0007FF0007FF002C
:1086000003FE0007FF0007FF000603000603000645
:10861000030006030006030006030006030007FF2D
:108620000007FF0003FE0007FF0007FF0007FF0031
:10863000006300006300006300006300006300004B
:108640006300007F00007F00003E0003FE0007FF84
:108650000007FF0006030006030006830007C300AF
:108660001F03003E030026030007FF0007FF00036F
:10867000FE0007FF0007FF0007FF00006300006324
:108680000000630000E30001E300036300077F00D4
:10869000067F00043E00040000031E0007BF000721
:1086A000BF000633000633000633000633000633EE
:1086B0000006330007F30007F70003F70000060089
:1086C0000003000003000003000003000003000794
:1086D000FF0007FF0007FF00000300000300000386
:1086E0000000030000030003FF0007FF0007FF0076
:1086F0000600000600000600000600000600000656
:10870000000007FF0007FF0003FF00000100000753
:1087100000000F00003E0000F80003E000078000AA
:1087200007000003C00000F000003C00001F000034
:108730000700000100000100000F00007F0001FCA5
:108740000007E00007800003E000007C00001F003D
:10875000001F00007E0003F80007C00007C00001F2
:10876000F800003E00000F000001000401000603B5
:1087700000070700038F0001DE0000FC0000780006
:1087800000F80001FC0003CE000787000703000685
:108790000100040000000100000300000700000FBA
:1087A00000001E00003C0007F80007F00007F8007A
:1087B000003C00001E00000F000007000003000046
:1087C000010006000007030007830007C30007E35A
:1087D0000006F300067B00063F00061F00060F00A0
:1087E0000607000603000FFF000FFF000C01000C3E
:1087F00001000C0100000100000700001C000070D7
:108800000001C0000E00000800000C01000C010077
:108810000C01000FFF000FFF00000200000300002A
:1088200001800000C0000060000030000030000047
:10883000600000C000018000030000020080000012
:108840008000008000008000008000008000008028
:108850000000800000800000800000800000000018
:10886000200000600001C0000100040000070000BB
:1088700007800001E00001F800019C00018C00016C
:108880009C0001F00001E0000780000600000400E9
:108890000007FC0007FC00066C00066C00066C007C
:1088A000066C00066C00066C0007FC0003BC0007A9
:1088B000FC0007FC00060C00060C00060C00060C71
:1088C00000060C00060C00079C00079C0007FC003B
:1088D00007FC00060C00060C00060C00060C000647
:1088E0000C00060C00031C0003F80001F00007FC5C
:1088F0000007FC00066C00066C00066C00066C00AD
:10890000060C00060C00060C0007FC0007FC00002B
:10891000CC0000CC0000CC0000CC00000C00000C0F
:1089200000000C0007FC0007FC00060C00060C0011
:10893000060C0006CC0006CC0006CC0006CC0007D6
:10894000DC0007DC0007FC0007FC000060000060A2
:108950000000600000600000600000600000600037
:1089600007FC0007FC0007FC0007FC0007C000072D
:10897000C000060000060000060000060000060019
:108980000007FC0007FC0007FC0007FC000060007B
:1089900000E00001F000019800030C00060C000646
:1089A000040004040004000007FC0007FC000600AB
:1089B0000006000006000006000006000006000099
:1089C00006000007FC0007FC0000380000700000F3
:1089D000E00001800003800000C00000700000186B
:1089E0000007FC0007FC0007FC0007FC0000180063
:1089F00000300000700000E00001C00001800003B2
:108A0000000007FC0007FC0007FC0007FC00060C48
:108A100000060C00060C00060C00060C00060C00FC
:108A2000060C0007FC0007FC0007FC0007FC000028
:108A30006C00006C00006C00006C00006C00006CAE
:108A400000007C00007C0007FC0007FC00060C0016
:108A5000060C00068C0007CC000F0C001E0C001644
:108A60000C0007FC0007FC0007FC0007FC0000CC22
:108A70000000CC0000CC0001CC0003CC0006CC00F0
:108A800006FC0004FC0004000006780006FC00065A
:108A9000CC0006CC0006CC0006CC0006CC0006CCF0
:108AA0000007DC0007D800000C00000C00000C00E0
:108AB000000C0007FC0007FC00000C00000C00008C
:108AC0000C00000C0007FC0007FC0006000006007C
:108AD0000006000006000006000006000007FC007B
:108AE00007FC00000400001C00003C0000F0000334
:108AF000C00007800007000003C00000F000003C39
:108B000000001C00000400000400003C0000F8000D
:108B100007C00007000003C000007800001C000030
:108B20007C0003E00007800007C00000F000003C6C
:108B300000000400040400060400070C0003980071
:108B400001F00000E00000F00001B800031C000686
:108B50000C00040400040000000400000400000CE9
:108B60000000180000300007E00007E000003000BF
:108B7000001800000C0000040000040004000006BF
:108B80000C00070C00078C0006CC00066C00063CAD
:108B900000061C00060C0006040000300000300037
:108BA0000078003FFFE07FCFF06000306000306071
:108BB0000030FFFFF8FFFFF8600030600030600019
:108BC000307FCFF03FFFE000780000300000300041
:108BD00000600000300000100000100000100000D5
:108BE00010000010000020000020000020000020E5
:108BF0000000200000300000100002000000030010
:108C0000060004000F000E001B000C0045000F00C2
:108C10006900100096000100C6000400C9000400AD
:108C2000D5000700E1000B00F60003001701050066
:108C3000200103002F01070038010C004D01040042
:108C400071010C007D010B00A1010E00C2010C009E
:108C5000EC010C0010020C0034020C0058020C0055
:108C60007C020300A0020300A9020C00B2020C0067
:108C7000D6020C00FA0209001E03130039030F008C
:108C800072030C009F030C00C3030D00E7030C00EC
:108C90000E040B0032040D0053040D007A0403008F
:108CA000A1040A00AA040E00C8040B00F2040E007E
:108CB00013050D003D050D0064050C008B050D002E
:108CC000AF050D00D6050D00FD050D0024060C00B6
:108CD0004B060E006F06120099060E00CF060F001D
:108CE000F9060C00260705004A070700590705008A
:108CF0006E070C007D070B00A1070400C2070D00E2
:108D0000CE070A00F5070A0013080B003108090016
:108D1000520809006D080B0088080B00A908020022
:108D2000CA080900D0080B00EB0809000C090C0068
:108D300027090B004B090B006C090A008D090B0079
:108D4000AB090B00CC090A00ED090A000B0A0A0066
:108D5000290A0C00470A0F006B0A0C00980A0C0045
:108D6000BC0A0A00E00A0800FE0A0200160B08000E
:108D70001C0B0E00340B00001803207E02000000C4
:108D8000FA8B00089C800008000000000BFE001E0B
:108D90000000001E01200F2001F0012E0F2001F025
:108DA000012E0120061C08221FFF08420882070C22
:108DB000003C00420C42023C010000C000200010B8
:108DC000078C08420840078007000C80085C086296
:108DD00008E20712061C09A0086008200400001E13
:108DE00007E018182004400240022004181807E089
:108DF000002400240018007E0018002400240040F5
:108E000000400040004007FC00400040004000409F
:108E100028001800010001000100010008000C00FA
:108E200003C00038000603F8040408020802040422
:108E300003F8000408040FFE08000C0C0A020902E3
:108E4000088208440C3808040802084208620452E8
:108E5000038C018001400120011801040FFE010074
:108E60000810081C08120812042203C203E0045868
:108E700008240822044203820004000200020C02BB
:108E800003820072000E071C08A20842084208A2D2
:108E9000071C0838084604820482034400F80820AE
:108EA00028201800004000A000A0011001100110AF
:108EB00002080120012001200120012001200120C1
:108EC00001200120020801100110011000A000A0E3
:108ED0000040000C00020B820062001C0FC010302A
:108EE00020084F0488C4882284128F1289E28832B5
:108EF0004404260811F00800080008000E0009C00C
:108F000001380106013809C00E00080008000802F7
:108F100008020FFE08420842084208640498030051
:108F200001F002080404080208020802080204040E
:108F3000021E080208020FFE0802080208020802C8
:108F40000404020801F0080208020FFE0842084269
:108F5000084208E20C060200080208020FFE08425E
:108F60000842004200E2000601F002080404080280
:108F7000080208020842084407CE0040080208021E
:108F80000FFE084208420040084208420FFE080255
:108F90000802080208020FFE080208020C0008027C
:108FA000080207FE00020002080208020FFE084243
:108FB000084200A001120A0A0C0608020800080272
:108FC00008020FFE08020802080008000C00020058
:108FD000080208020FFE080C083001C002000E0053
:108FE00001800870080C0FFE08020802080208023F
:108FF0000FFE08080810002000C0010202020FFE48
:109000000002000201F0020804040802080208023B
:1090100008020404020801F0080208020FFE088298
:10902000088200820044003801F0020804040802AB
:109030000802180228022404420841F0080208022B
:109040000FFE0842084200C203240418080008006A
:109050000E1804240822084208420484030E000E5D
:109060000002080208020FFE080208020002000EB9
:109070000002000203FE04020802080008020402C3
:1090800003FE0002000200020002001E00E20700D0
:109090000800070000E2001E0002000200020002B9
:1090A000000E007203800C020382005E00E20300E7
:1090B0000C0003E2001E00020002080208020C0677
:1090C0000A0A01B2004001B00A0A0C0608020802AE
:1090D00000020002080E08320FC00820081A00061D
:1090E0000002000208000E0E09020882086208123F
:1090F000080E0C0202007FFE4002400200060078CB
:1091000003800C00400240027FFE00400030000C53
:1091100000020002000C003000404000400040000F
:10912000400040004000400040000002000C0E40A3
:109130000920092004A00FC00800000407FE084011
:10914000082008200440038007C0082008200820C9
:109150000440038004400820082004440FFE04005B
:1091600007C008A008A008A004C008200FFC08221F
:1091700008220002000430004DC04A204A204A2044
:1091800049E0302008040FFE0840002008200FC0EE
:10919000080008400FE208004000400040403FE265
:1091A00008040FFE0900018006600820082008005E
:1091B00008040FFE080008400FE0084000200820C7
:1091C0000FC00840002008200FC0080008400FE032
:1091D0000840002008200FC0080003800440082039
:1091E00008200440038040407FE0444008200820DD
:1091F00004400380078008400820082044407FE0A6
:10920000400008400FE00840002000200CC009206A
:109210000920066000200FF808200420002007E045
:109220000800080004200FE00400002000E00720F0
:109230000800072000E00020002000E007200C00CC
:10924000032000E007200C00032000E0002008209D
:109250000C600AA001000AA00C600820402040E039
:1092600023201C00072000E0002008000C600B20D9
:1092700008A008600C2000801F7820044002FFFE38
:10928000400220041F7800800100008000800080E0
:109290000100010001000100008002000000010047
:1092A00004000300060008000C0006001C000C006F
:1092B00028000B0040000100560004005800040084
:1092C00060000700680009007600020088000400C2
:1092D0008C00010094000400960006009E0004002B
:1092E000AA000600B2000600BE000700CA00060081
:1092F000D8000600E4000700F0000600FE000600AB
:109300000A01010016010200180107001C010900F2
:109310002A0107003C0105004A010E0054010B0020
:10932000700109008601090098010A00AA010900DC
:10933000BE010800D0010A00E0010B00F4010500A5
:109340000A02060014020B002002090036020E0079
:1093500048020C0064020A007C02080090020A0025
:10936000A0020A00B4020700C8020900D6020B00DE
:10937000E8020B00FE020F0014030B0032030A0088
:10938000480309005C0303006E0304007403030038
:109390007C0308008203080092030200A203060077
:1093A000A6030700B2030500C0030700CA030500B7
:1093B000D8030600E2030700EE030700FC030300E6
:1093C0000A040400100408001804030028040B0019
:1093D0002E04070044040600520407005E04070040
:1093E0006C0405007A040400840404008C04070063
:1093F00094040700A2040B00B0040700C604070091
:10940000D4040600E2040400EE040100F6040400A3
:10941000F8040900000500000E02207E0200000092
:109420009A920008888D00080000000013F00038B0
:1094300000000000003802001E8003801EF0038040
:1094400002F00280008010E011903FF813100E101F
:1094500010600890049003600D80124012200C10E0
:109460000E00190011E0119016901C601C00030002
:1094700000380FC01860201040084008400840081D
:10948000201010200FC0002001C000B0008001C0DB
:1094900000200200020002001FC0020002000200C1
:1094A0005800380002000200020002000200020020
:1094B000180018004000300008000600018000403D
:1094C0000030000807C0182010101010182007C026
:1094D0001020102010101FF01000100010001810A5
:1094E00014101210111010E0101011101110129021
:1094F0000E600600050004C004201FF0040010F0F8
:10950000109010900F1007C009201090109010902C
:109510000F000010181006100190005000300E606F
:1095200011901110111013900E6001E01210121022
:109530001210092007C018C018C058C038C0020057
:1095400002000500088008801040050005000500A5
:109550000500050005001040088008800500020095
:10956000020000300010121001100090006007C0CF
:10957000086013B014D014501A5007E00400100013
:109580000C0007800460046007800C0010001FE0DE
:1095900011201120112011200EC00780084010203A
:1095A00010201020102010201FE01020102010206C
:1095B000084007801FE012201220122012201020E5
:1095C0001FE0022002200220022000200780084025
:1095D00010201020122012201E201FE00100010088
:1095E000010001001FE0102010201FE010201020BB
:1095F00010001020102010200FE01FE001000300D9
:109600000480084010201FE010001000100010001F
:1096100010001FE0006003800400038000601FE072
:109620001FE000400180060008001FE0078008409E
:10963000102010201020084007801FE00220022088
:109640000220022001C007800840102010201020B6
:109650002840678040001FE002200220062009C049
:10966000100010C011201120112012200C20002009
:10967000002000201FE00020002000200FE010004C
:109680001000100010000FE0002001C00E001800B4
:109690000C00030000C0002000E00F001C0003804D
:1096A000070018000F8000601020084004800300AD
:1096B00003000480084010200020004001801E00AC
:1096C00001800040002010201820142012201120BA
:1096D00010A010607FF840084008400800080030E3
:1096E00000400180060008003000400040084008AB
:1096F00040087FF80400030000C0007003800400ED
:109700002000200020002000200020002000200059
:10971000000800100C001240124012401F80100080
:109720001FF808801040104010400F80070008808C
:1097300010401040104010400F801040104010406A
:1097400008801FF80F0012C0124012401240138010
:10975000004000401FF000480048004800480F80CB
:1097600090409040904088807FC01FF8008000406B
:10977000004000401F800040004000581FD880403B
:10978000804080587FD81FF80200050008801040F4
:109790000008000800081FF81FC0008000401FC01C
:1097A000008000401FC01FC00080004000400040FB
:1097B0001F800F8010401040104010400F80FFC0ED
:1097C00008801040104010400F800F801040104063
:1097D00010400880FFC01FC000800040004000C053
:1097E00011801140124012400C40004000400FE038
:1097F0001040104010400FC0100010001000080072
:109800001FC0004003800C0010000C0003800040CB
:1098100000C007001C00038007001800070000C0FC
:1098200010400880070007000880104080408180B9
:10983000C600780018000600018000401040184063
:1098400014401240114010C0010001003EF84008D1
:1098500040087FF8400840083EF001000100040085
:1098600002000200020004000400040002000200E2
:109870000000010004000400060008000E000500BE
:109880001E000800280008003800010048000500FC
:109890004A000500540006005E0007006A0002004E
:1098A000780006007C000200880008008C0006009A
:1098B0009C000700A8000500B6000500C0000600D7
:1098C000CA000400D6000600DE000600EA0006001A
:1098D000F6000600020102000E010200120106005D
:1098E00016010600220106002E0106003A010800BA
:1098F00046010800560106006601070072010600D5
:10990000800106008C01060098010700A4010600F2
:10991000B2010500BE010500C8010600D201060023
:10992000DE010700EA010600F80107000402060054
:10993000120208001E0206002E0206003A0207006C
:109940004602060054020800600208007002080087
:1099500080020700900207009E020400AC0208008B
:10996000B4020400C4020600CC020800D8020200BF
:10997000E8020600EC020600F802060004030600F6
:10998000100306001C030700280306003603060028
:10999000420304004E030400560305005E03040066
:1099A00068030700700306007E0306008A030600B2
:1099B00096030600A2030500AE030500B8030600E7
:1099C000C2030600CE030700DA030800E80306001E
:1099D000F803080004040600140405002004010034
:1099E0002A0405002C040800360400000B02207E27
:1099F000020000006E9800082894000825686400A2
:109A00004C7620555000000000004C7620444E005B
:109A1000000000002052697365000000000020462D
:109A2000616C6C0000000000494E2057696E000018
:109A300000004F55542057696E0000002053796E86
:109A4000632042002053796E63204100302E312084
:109A5000562F44697600302E3220562F4469760006
:109A6000302E3520562F44697600312E3020562F67
:109A700044697600322E3020562F44697600352E08
:109A80003020562F446976003530306E732F44698C
:109A900076003175732F4469760000003275732F9C
:109AA0004469760000003575732F44697600000024
:109AB000313075732F4469760000323075732F444E
:109AC00069760000353075732F44697600003130B7
:109AD0003075732F4469760032303075732F4469C6
:109AE000760035303075732F44697600316D732FF1
:109AF000446976000000326D732F446976000000DF
:109B0000356D732F44697600000031306D732F443A
:109B10006976000032306D732F44697600004E4F35
:109B20004E450000000000004E4F524D0000000066
:109B3000000053494E470000000000004F46460019
:109B40004143200044432000484F4C4400000000A3
:109B500052554E0052616E67653A00004368616E6F
:109B60006E656C20420000004368616E6E656C207B
:109B70004100000080004000C0002000A000600004
:109B8000E000100090005000D0003000B0007000E5
:109B9000F000080088004800C8002800A8006800FD
:109BA000E800180098005800D8003800B800780085
:109BB000F800040084004400C4002400A4006400F1
:109BC000E400140094005400D4003400B400740085
:109BD000F4000C008C004C00CC002C00AC006C009D
:109BE000EC001C009C005C00DC003C00BC007C0025
:109BF000FC00020082004200C2002200A2006200BB
:109C0000E200120092005200D2003200B200720054
:109C1000F2000A008A004A00CA002A00AA006A006C
:109C2000EA001A009A005A00DA003A00BA007A00F4
:109C3000FA00060086004600C6002600A600660060
:109C4000E600160096005600D6003600B6007600F4
:109C5000F6000E008E004E00CE002E00AE006E000C
:109C6000EE001E009E005E00DE003E00BE007E0094
:109C7000FE00010081004100C1002100A10061003F
:109C8000E100110091005100D1003100B1007100DC
:109C9000F100090089004900C9002900A9006900F4
:109CA000E900190099005900D9003900B90079007C
:109CB000F900050085004500C5002500A5006500E8
:109CC000E500150095005500D5003500B50075007C
:109CD000F5000D008D004D00CD002D00AD006D0094
:109CE000ED001D009D005D00DD003D00BD007D001C
:109CF000FD00030083004300C3002300A3006300B2
:109D0000E300130093005300D3003300B30073004B
:109D1000F3000B008B004B00CB002B00AB006B0063
:109D2000EB001B009B005B00DB003B00BB007B00EB
:109D3000FB00070087004700C7002700A700670057
:109D4000E700170097005700D7003700B7007700EB
:109D5000F7000F008F004F00CF002F00AF006F0003
:109D6000EF001F009F005F00DF003F00BF007F008B
:109D7000FF000400000800000000000000020001D5
:109D80000000100002400000000000A000000000E1
:109D900005400000000000C8000000000C4000006A
:109DA0000000409C00000000194000000020BCBEE4
:109DB0000000000034400000BFC91B8E00000004FA
:109DC000B5400000504BCFD06607E2CF0100000045
:109DD0006C4100003E8251AADFEEA7340100000072
:109DE000D9420000DCB5A0E23A301F97FFFFFFFF29
:109DF000B4450000FD25A0C8E9A3C14FFFFFFFFF48
:109E0000FF3F00000000008000000000FF3F000056
:109E10000000008000000000422E4C2E383000630D
:109E20006F7272205A2041006F666673657420411C
:109E300000636F7272205A2042006F666673657409
:109E4000204200696E74657270002053796E632041
:109E500041004C7620555000506F73205800482028
:109E6000204C6576656C004C20204C6576656C0056
:109E7000437572736F723100437572736F72320083
:109E80004D31004D32004143004E4F4E450054527B
:109E900049470052554E004D454E5500352E302055
:109EA000562F446976003530306E732F4469760042
:109EB000436F72726563742044697620436F6566F0
:109EC0006600536176652053657474696E6773200C
:109ED000746F20666C617368004175746F20436F06
:109EE0007272656374696F6E205A65726F00436F9A
:109EF0006C6F727300557365722050726573657470
:109F00007300457869740000449F00080000002039
:109F10005C1000002801000810A100085C1000205F
:109F20009C060000840100081C00000043000000A3
:109F3000F8FFFFFF0C0000000E0000000F00000003
:109F40002E00000031600801014001010120137D55
:109F5000176508900101590761234108167F7E5952
:109F6000CEC81278120A148F01DC121423419B9A76
:109F700080011931220B138545192C2106FFA0EB16
:109F80009B059001FF01FF01FF01FF01FF01470653
:109F9000FFBD0341059201FF01FF01FF01FF01FF2A
:109FA000014713020322FF123212FA6A2001013A1A
:109FB000293D45020406082D010203040475060725
:109FC00008091201120212031204120512061405E6
:109FD0000550143C01C31250120F1E2108A0EBFFC4
:109FE0008613189E3D083C01AA14114A50143A1FCA
:109FF000143A96144BBD03143A3114BA7D283A280A
:10A0000014BA69283A3A143A1E144B6001141A43E0
:10A010001419A7100D422E4C2E2038302020040495
:10A02000782B718C04221422F813EA0D3D203C0198
:10A0300078344BA0A9343A5848BA5F483A5214BA17
:10A040004B283A4A14BA32280A115E841A6714411E
:10A05000143201309A5A181A70181A322CA9145A4C
:10A06000782C81120112059A26201A97201A291499
:10A070001A4914114A50141A9C145A74145AE42898
:10A0800029141ABF149A4B3C1AA614140C01059AF1
:10A0900028141A8E14DA36141A89141A60149A17AE
:10A0A000141A8014DA79141A83141201BADC3C1AD7
:10A0B00093141A2B149A1EA01A86145A4B1469A0D2
:10A0C00029141A6E142ABE281149145AAFFC23050C
:10A0D000051A0F1A1AAA0627BD03A0EB60011AEE93
:10A0E0001C1A0F12A9143AD914BA96143AB014BA19
:10A0F00082143AF514BA6E143AC2143A5A1429A8C2
:10A100001122F84B029F80011519A00138000000B0
:04000005080000ED02
:00000001FF
